:020000040000fa
:08000000c01404000000000020
:020000040000fa
:1000080004140000081400000c1400001014000070
:1000180014140000bc140000bc140000bc14000040
:10002800181400001c140000201400002414000000
:10003800bc140000281400002c1400003014000028
:1000480034140000381400003c1400004014000070
:100058004414000048140000bc140000bc14000044
:100068004c140000501400005414000058140000f0
:100078005c140000bc140000bc140000bc14000098
:10008800bc14000060140000641400006814000030
:100098006c14000070140000741400007814000040
:1000a8007c14000080140000bc140000bc14000084
:1000b800bc14000084140000881400008c14000094
:1000c800bc14000090140000bc140000bc14000014
:1000d800bc14000094140000bc140000bc14000000
:1000e800bc140000981400009c140000bc1400000c
:1000f800bc140000bc140000bc140000bc140000b8
:10010800bc140000bc140000bc140000bc140000a7
:10011800bc140000bc140000a0140000bc140000b3
:10012800bc140000a4140000a8140000ac140000c3
:10013800bc140000bc140000bc140000bc14000077
:10014800b0140000bc140000bc140000bc14000073
:10015800bc140000b4140000bc140000bc1400005f
:10016800bc140000bc140000bc140000bc14000047
:10017800bc140000bc140000b8140000bc1400003b
:10018800bc140000bc140000bc140000bc14000027
:10019800bc140000bc140000bc140000bc14000017
:1001a800bc140000bc140000bc140000bc14000007
:1001b800bc140000bc140000bc140000bc140000f7
:1001c800bc140000bc140000bc140000bc140000e7
:1001d800bc140000bc140000bc140000bc140000d7
:1001e800bc140000bc140000bc140000bc140000c7
:0801f800bc140000bc1400005f
:020000040000fa
:10280000c014040000000000d66b040000000000ab
:10281000d66b040000000000d66b0400000000002e
:10282000d66b040000000000d66b0400000000001e
:10283000d66b040000000000d66b0400000000000e
:10284000d66b040000000000d66b040000000000fe
:10285000d66b040000000000d66b040000000000ee
:10286000d66b0400000000005a6a0400000000005b
:10287000d66b040000000000d66b040000000000ce
:10288000d66b040000000000d66b040000000000be
:10289000d66b040000000000d66b040000000000ae
:1028a000d66b040000000000d66b0400000000009e
:1028b000c84a040000000000d66b040000000000bd
:1028c000d66b040000000000d66b0400000000007e
:1028d000d66b040000000000d66b0400000000006e
:1028e000d66b040000000000d66b0400000000005e
:1028f000d66b040000000000d66b0400000000004e
:10290000d66b040000000000d66b0400000000003d
:10291000d66b040000000000d66b0400000000002d
:10292000d66b040000000000d66b0400000000001d
:10293000d66b040000000000d66b0400000000000d
:10294000d66b040000000000d66b040000000000fd
:10295000d66b040000000000d66b040000000000ed
:10296000d66b040000000000d66b040000000000dd
:102970007c6b040000000000d66b04000000000027
:020000040000fa
:102980004f7421000e7f22000e018800000000001d
:1029900000012000200288000c00070040522600a1
:1029a0000100200011000700000020000000e000ee
:1029b000020032000000020000000000d8670200a0
:1029c000000000000040da000000fe004440a900c2
:1029d000c06320000000e00003003200000020007f
:1029e000a00188004440a800000006009101880072
:1029f000800078000000eb0015003700e280400006
:102a000032a0b4009101ba00e280400032a0b400cc
:102a10009102ba00e280400032a0b4000002eb0054
:102a2000472bde00f507b200602ce10004003a00fd
:102a30000059eb008301e900fdff3e000400370070
:102a40006128e100010032000082eb000400070071
:102a50001101ba000200e000e8ff3a0000000600a1
:102a60003159ba008301e9000c0032002159ba0043
:102a70008301e900080032000400e00003003a008e
:102a8000e280400032a0b400f5ff370011d9ba004f
:102a90008301e900faff3a008100e800e18040008c
:102aa00032a0b4000000060000000000000000009a
:102ab0000000000000000000000000000000000016
:102ac0000000fa0016a2a9001682a8000080fa00f1
:102ad000000006000000fa0000000000b4108000b2
:102ae00061026200e00f5200fcff3a00b410800067
:102af00062026200e00f5200f8ff3a00b41080005a
:102b000064026200e00f5200f4ff3a00b41080004b
:102b100068026200e00f5200f0ff3a00b41080003b
:102b200070026200e00f5200ecff3a00c510800016
:102b30000400240004826200e00f5200e7ff3a0024
:102b40000080fa00000006000000fa001662a800eb
:102b500000000000b410800068026200e00f520024
:102b6000fcff3a0018c2a9008410800004427800db
:102b7000044078000080fa00000006000200fa001d
:102b8000004f78009e4278000582fb009410880078
:102b9000c51080000408200004826200e00f52008b
:102ba0000200320000c2eb00010037000042eb00df
:102bb000044078000080fa00000006000000fa00df
:102bc00016a2a8001682a8000080fa0000000600e5
:102bd0000400fa00000f7800110798001e02900010
:102be000a41088001e027800b41088000080fa004b
:102bf000000006000000fa001602a8000080fa009b
:102c0000000006000000fa001642a8000080fa004a
:102c100000000600839f68000100e00002003d0004
:102c200060001000e08018000300e00002003d009a
:102c300060011100e0811900050007004f00e0006d
:102c400002003b0060001000e08018000000060059
:102c50006022b800060220000000d0008180d2006f
:102c60000482d2008582d2000000a000020252003d
:102c700083825a00030031000202420083824a002c
:102c80000000a1000603e900f3ff3a00000006007f
:102c9000e4874700889fbe008a9fbe008c9fbe00cd
:102ca0008e1f780024b72000955b8000e08f5200d3
:102cb0000b003a00e4024200955b8800e55b880067
:102cc00024029800d45b8800a44290000504a00070
:102cd00025429800e44290000504a0006542980057
:102ce000670440004244de004244dd00d25b8000c5
:102cf000c4b82000497421008484540025002000b9
:102d0000110009008504d80080bf9f00050744001a
:102d10000e0747000003eb00e40544007c7421002b
:102d20000406560008064600020037001600200080
:102d30000d01780022429000610262000200320020
:102d40000a003700150978009202780025429000a9
:102d500061026200fbff320008024100848f5200d2
:102d600002003900e00f54003f003d009206780059
:102d70000d00a100828f5600edff3e00e10f5300d1
:102d8000eaff3a000fba9700840f540002003600a1
:102d9000890f5400100039006143b800614ab9003e
:102da000b0ff2f000100200004025000858258006f
:102db000840f5300858f5b00020035000b057800ff
:102dc00006003700110009000986d8000982b90001
:102dd00004057800010037000e0578000a0078002d
:102de000db030700e10f400005003a000b05780007
:102df0000b007800d6030700e10f40002b003200e3
:102e0000e45b8000000a7800e45b80006403420019
:102e1000a4429000860f5000020032000504a0007a
:102e2000010037000504a100254298006405550003
:102e30000a0540000a087800ea5b880024b72000f1
:102e4000040d7800e55b8000254290000404a0009a
:102e5000a4429800204290000404a100244098005d
:102e60000003eb00b2ff3700d45b8800848f520070
:102e7000070036001403be00f65b8800075c88007c
:102e8000120a78008042eb00d45b80002542980053
:102e9000d75b800007097800224290000404a0005c
:102ea0002441980064004100010037000000eb005d
:102eb0004f0778004f06be004f05be004f04be000e
:102ec0004f00b10000000600e00f50000800320083
:102ed00064005000d45b8000840f5000010031007a
:102ee000d05b8800204290000404a1002440980098
:102ef00000000600889fbe008a9fbe000004be003e
:102f0000e08f540005003a00e00f54003200320018
:102f100008007800ecff070030003700e00f540095
:102f200004003a000900780059ff07008004780087
:102f30002a003700640254009405780068fa97006c
:102f4000610262000200320008007800deff070024
:102f5000090078004eff070080047800e08f5400dd
:102f60001e003200888f54001b00320069bd97009c
:102f70000905550042d5de0088855500c2ddde001a
:102f80000a0178008b0f5500010036000b01780014
:102f90004211dd0088007800090078001300070066
:102fa000888f54000d0031004255dd000a85440031
:102fb000880f5500090036000804550042c4de00a1
:102fc0004244dd0008844400f45b8000055c80001e
:102fd000048cbe00010037008804780009007800e6
:102fe0004f05be004f04be0000000600000278003e
:102ff00002003700315a78000201e900e00f510069
:10300000fcff3a00000006000c00fa00889fbe009a
:1030100000047800f4ff2700d4bf9f008004eb0079
:1030200099bf9f0088bf9f00a8bf9f00240c20006d
:10303000b4bf9f0078815700cfb0970070805700d1
:10304000070007000fba9700094a78000fba9700e7
:10305000080052004f04be000080fa000000060085
:103060002f03b000889fbe008a9fbe008c9fbe00c9
:103070008e1f7800e0af9f00c1af9f00b2b79f00e6
:103080008006eb006e023700cfa897008100e800b1
:10309000c1af9f0054c2b300844f500006003a00f5
:1030a000010278000006eb0001c3b30000c2b300c8
:1030b000b7c2b300070037000000fb00efa897007d
:1030c0006b020700e10f40005d0232008d06e80050
:1030d0005b0237008402780034437800d2c2b30028
:1030e000824f53000900320005003c00804f53001e
:1030f00008003200874f53000c003a0007003700e9
:10310000814f530009003a00060037000c30a00040
:10311000f0ff37000c00a000eeff37000c10a000fd
:10312000ecff37000c20a000eaff370062026600c7
:10313000010032000c00a1006802660001003200ac
:103140000c20a1000602fb000403b100e90f5200ad
:103150000c003e00050378000002eb006a22b90073
:10316000b603fb000703b100048243008602780027
:103170009603fb000703b100e98f5300f7ff360009
:10318000080037000002eb00a7c2b300874f5300ce
:1031900004003a00bfb1970043027800b3b79f0024
:1031a0008502e8000007eb00e6c2b300954f13006c
:1031b0000a003a000ce0a00064435300d54f13000e
:1031c0000200320005037800080037003fb3970083
:1031d00046077800b6b79f008502e800050378002f
:1031e000080037006a70b900008743008602780043
:1031f000b603fb000703b100e98f5300f9ff360067
:10320000f6ff3700b6427800c6af9f00c0c6b300d5
:1032100080cf5200250032000f003c0036c6b300bc
:1032200086cf52006e00320004003c00e0cf520016
:10323000080232006b4353000f00370046c6b3004c
:1032400086cf5200170032006543430086cf5200fc
:1032500083003a001300370036c7b30086cf520010
:103260001f00320007003c006443530086cf520029
:10327000140032000643e80086cf520078003a007e
:103280001300370056c7b30086cf520079003200d2
:103290006343430086cf520071003a00a5c79f00e8
:1032a0000d003700a5c79f0074003700f0036600cb
:1032b0000501200001003200050028000506760007
:1032c000d0ff3700a5c79f000c60a0006b0037003f
:1032d000a5c79f000c50a0000c70a000670037002d
:1032e000a5c79f00bfb09700c1027800b1b79f008b
:1032f00005047800e08f520001003a0048b4200035
:10330000080378008002eb00010037008502e80026
:10331000e6c37a00e0cf5300fcff3a008504780052
:10332000e00f570003003200890f57000100310001
:103330008e0478000007eb00890f52000100360070
:10334000090752006806660014003a0007003700bb
:10335000efa8970000022000c5010700e10f400020
:10336000010032008d06e8000e07e900e00f57006b
:10337000f7ff3a000087eb000800370008027800ea
:103380003400fb0004047800efa89700b8010700a0
:10339000e10f4000010032008d06e80009027800cc
:1033a0008404e900e00f5200f4ff3a00e00f5600f9
:1033b000a301320007003700efa8970000022000a9
:1033c000ab010700e10f4000010032008d06e8006c
:1033d0000e07e900e00f5700f7ff3a0098013700a9
:1033e0003fb19700c2027800b2b79f000500780095
:1033f000cf80de000101780082017800f0af9f00ed
:1034000081b79f0092b79f00a3b79f004800de00de
:10341000c80add0000807200a0c79f00700366002c
:1034200009003200e04f500007003200e14f400039
:1034300005003200b0c79f006fdb9700c6c79f0032
:103440002900200003003700efdb9700b7c79f007b
:103450001900200038fc2f000f044400b0ff370093
:10346000a5c79f0028fc2f000f044400190020006e
:10347000abff3700a5c79f000c0cb3008c0278008f
:10348000050cb2002b003a00e00f560005003d008d
:103490003fb097004005be004004be00b0b79f009b
:1034a00017003700f00266000f003200bfb297002d
:1034b0004501be00b5b79f00c2a79f00d3a79f00dc
:1034c0000503780096029000cfaade00e5a79f00d2
:1034d000f5a79f004fa49700dfa497006fa5970062
:1034e000ffa59700060037003fb097004004780022
:1034f000b0b79f00cfc4de00090578008a057800c8
:10350000e00f5400e08f5c00e00f5d00e08f5d0095
:1035100025003d003c00b3006000b8006011b80019
:1035200008045000898458000a0559008b85590009
:103530001d003700e00f560005003d00bfb09700aa
:103540004105be004104be00b1b79f001600370020
:10355000f00266000e003200bfb297004501be00c7
:10356000b5b79f0082af9f0093af9f000003eb00b1
:10357000a6af9f008003eb00b7af9f000fac970092
:103580009fac97002fad9700bfad970006003700a6
:103590003fb0970040047800b0b79f0009002000ba
:1035a0000a0020000b002000e00f570007003a003f
:1035b0001e002000e00f5400e08f5c00e00f5d0073
:1035c000e08f5d00010032000007eb008c00780006
:1035d000010cb200f1af9f0005042000858f500060
:1035e0002c00320003003c00e08f50000800320045
:1035f0003c003700050820007fa99700850f510087
:1036000010003200050c2000850f510035003a00f3
:10361000a6a8200015c0b3003600be003601be00cb
:103620000040e10001c8e10002d0e10003d8e10060
:103630002b0039008542e800f4cf5200f6ff3a0033
:103640002700370015c0b300000120000100200052
:103650006011b8000040e10001c8e10002d0e100c3
:1036600003d8e1001e003900460020000000d00011
:103670008180d2000281d2008381d2000603e9005a
:10368000faff3a008542e800f0cf5200f1ff3a001d
:103690001300370015c0b300800020000100200097
:1036a0006011b8000040e10001c8e10002d0e10073
:1036b00003d8e1000a003900370020000000d000e4
:1036c0008180d2000281d2008381d2008703e90089
:1036d000faff3a008542e800f5cf5200f1ff3a00c8
:1036e000a5c79f002fc097008002fb008e8f52005d
:1036f00002003d00aec79f0003003700850f570052
:1037000001003d0005077800e00f52000300320081
:10371000e3026600010032000402e9000500240013
:1037200085026600050032008e0f52000200340050
:103730000e025200010037000002eb002fc197007b
:103740008202fb008001eb00d3af9f00850f520087
:103750000200340085025200d5af9f00640266006b
:103760002c003200e202660061026600e08f520027
:1037700006003200b0022000e00f520001003200cb
:103780000080e800efa8970004003700e00f520027
:1037900006003200efa8970000022000b4000700e6
:1037a000e10f4000010032008d06e8005faa97009b
:1037b000e00f52008d0032000802be000a03be0076
:1037c000dfac9700efa8970000032000c4b79f006c
:1037d000d5b79f00e6b79f00f7b79f00a40007008a
:1037e0004fb29700dfb297006fb39700ffb3970017
:1037f000e10f4000010032008d06e8008904e90075
:10380000f0ff3a00d9af9f000605be000404be00d9
:1038100076003700dfaa9700e08f520018003200d0
:103820006802660016003a000802be000a03be00e5
:10383000dfac9700efa8970000022000c4b79f00fc
:10384000d5b79f00e6b79f00f7b79f008800070035
:103850004fb29700dfb297006fb39700ffb39700a6
:10386000e10f4000010032008d06e8008904e90004
:10387000f0ff3a00d9af9f000605be000404be0069
:10388000e202660061026600e08f5200060032002c
:10389000b0022000e00f5200010032000080e8007a
:1038a000efa8970004003700e00f52004f003200ed
:1038b000efa89700000220006d000700e10f400014
:1038c0004a0032008d06e800480037000e07e90084
:1038d0007fab970007042000870f53002d003200b4
:1038e00003003c00e00f53000800320037003700af
:1038f000040820007fae9700840f560012003200ab
:10390000040c2000840f560030003a004372dd00a2
:1039100020a82000000242005403be004402be0062
:103920000800be000a01be00d6010700a400200066
:10393000050020006033b800d901070004c3b300bc
:10394000044240002000370034b32000bfa297009b
:10395000e08f52000100320024b22000c272dd006c
:103960000800be000a01be008502e9000500330020
:103970008301d1000281d3008180d3000080d30075
:10398000f9ff37006f00600064407800a0c79f0017
:103990000e0037006372b9000800be000a01be00c5
:1039a000040678000c06e900050033008301d1000d
:1039b0000281d3008180d3000080d300f9ff37005b
:1039c000674260000443b000a4c79f00afc09700e7
:1039d0000100fb00efa8970025000700e10f400061
:1039e000060032008d06e800040037000c01780064
:1039f0000202b200b2a79f008cbf9f00e00f5700e9
:103a0000b2ff3a000fbe9700680666000c00320055
:103a1000dfa99700e08f5100090034000306780009
:103a2000efa897000002200011000700e10f4000fe
:103a3000010032008d06e8000c06e900f8ff3a00ac
:103a40004faa970014407800a0c79f00e04f500095
:103a50008dfd3a000d0078004f0778004f06be003c
:103a60004f05be004f04be002f03b100000006004a
:103a7000889fbe000104780038029000e2026200d4
:103a80008084eb003b003200040378000620b20083
:103a90009802900002003a00e08f520035003a0090
:103aa0000490a0003404980080047800f90fb2005c
:103ab000e08f520002003a00a8029000050c780046
:103ac000ea8f540005003a000408b20003003a00ef
:103ad00088007800d0002000e5ff07001802900061
:103ae000d8029000850f52000b0032000402e8005b
:103af0001404980018027800094a7800040ce800c1
:103b000015c0b30024b82000054a7800ea8f54009d
:103b100018003a0005003700880078000940780056
:103b20001700070080047800120037003802900068
:103b30000410b2000f00320018019000a80090009d
:103b4000480090005200070018029000840f5000b7
:103b500004003200380290000403b30034049800db
:103b60008084eb000002eb0014049800280290000f
:103b7000040c7800090078004f04be000000060025
:103b80000200fa00889fbe00a0ff9f000104780099
:103b900038029000840278000504b200020032006e
:103ba0000000fb0035003700e202620005003a0029
:103bb0000403b30034049800150498000080eb005f
:103bc0002e003700d8049000e08f540006003a0021
:103bd00012002000e6805700480090002c000700eb
:103be0001904980023003700a8029000e08f5200cb
:103bf00008003a0055b8200025049800050c78000c
:103c00002500200055049800150498000430a000f9
:103c10003404980018019000a8009000480090001b
:103c20001b000700280290008082eb00150498001a
:103c3000affa9700054a7800040ce8002ffa9700c5
:103c4000ea4f52000b003a00380290000410b20014
:103c50000800320018019000a80090004800900071
:103c60000b0007000002eb0014049800a80290006b
:103c7000050c78002ffa97000400fb004f04be00eb
:103c80000080fa000000060000c0da000000060014
:103c90000a00fa00e20f500022003e00445c80005f
:103ca000e10f520006003200872320004623200047
:103cb0002423200005232000e08f530004003a0055
:103cc00087222000462220002422200005222000f6
:103cd000000028001500600003003a00800b780007
:103ce00007002800958a7300054020009482620036
:103cf00001003a0014a0a0008202780006003700fc
:103d0000940378000710b200fdff3200b103fb00fe
:103d1000070b78008502e900e08f5200f8ff3a00b7
:103d20000800370034002000b4bf9f00c0bf9f00d0
:103d3000d1bf9f00e2bf9f006a805700d2ff0700fb
:103d40006fb99700020078000080fa0000000600ba
:103d5000889fbe0080047800505c8000e00f500017
:103d600004003a000e0007000084eb00e00f500052
:103d700008003500585c8000e08f540005003200d8
:103d80000900440006000700e00f500001003d005c
:103d90000084eb00080078004f04be00000006001d
:103da000e00f500004003a00c4b82000545c8800c2
:103db00000027800060037000082eb004574210005
:103dc000850f500002003e00505c88000002eb00ae
:103dd0000400780000000600889fbe008a9fbe0095
:103de0003004be002005be000404440085844c005d
:103df00006054d0087854d000898be000a90be005c
:103e00000440e10005c8e10006d0e10007d8e10068
:103e100002003100680040001008e8004f05be00b5
:103e20004f04be00000006001000fa00889fbe008c
:103e30008a9fbe000605be000404be003002be001c
:103e40002003be00c4b79f00d5b79f00e6b79f0010
:103e5000f7b79f000802520089825a000a035b00ec
:103e60008b835b0084bf9f0095bf9f00a6bf9f0010
:103e7000b7bf9f000498be000698be001100200046
:103e80004fb29700dfb297006fb39700ffb3970070
:103e90000820e10009a8e1000ab0e1000bb8e10048
:103ea000010039008000eb00108810004f05be00b3
:103eb0004f04be000080fa00000006001400fa0063
:103ec000889fbe008a9fbe008c9fbe003f000700f7
:103ed0000605be000404be000006eb00ccb79f0040
:103ee000bcb79f00acb79f009cb79f008cb79f00ea
:103ef0000d0420004fb39700bfb297008603430024
:103f00002fb29700e00f530004003d003d00070072
:103f10000f004000b0ff0700030037003900070022
:103f20000f004000c0ff0700cfb2970095bf9f0071
:103f3000e08f5200090035002b000700140020001c
:103f4000050020006033b80000007200818072001c
:103f500002017300838173001c0007000c06e80057
:103f60008d0f5600e3ff3a001fba9700e00f520092
:103f700005003d000802be000a03be0000fe2f003f
:103f80000f00400094ff07004faa9700e00f520077
:103f900008003a000fb497009fb497002fb5970020
:103fa000bfb59700d8b79f00e9b79f00fab79f0049
:103fb0008bbf9f000c0007004f06be004f05be00e0
:103fc0004f04be000080fa00000006000100070058
:103fd0000000060090b79f00a1b79f00b2b79f00f6
:103fe000c3b79f00000006000100070000000600a4
:103ff0001fb09700afb097003fb19700cfb19700c7
:10400000000006004f2bde0087037300a7b79f0058
:104010004f23de00858242008502730095b79f0022
:10402000ffaa97004f2bde00040242000402730037
:1040300084b79f006faa97004f23de00858242005d
:1040400085027300f5af9f00e9ff07004f18de00ff
:104050000402420000027200e4af9f00e4ff070088
:10406000000040008180480002014900838149002e
:10407000d8ff07000802be000a03be0000fe2f00a2
:1040800000000600881f780018002000881f7800b4
:104090008aff07008f87e9004f04780000000600c0
:1040a000801feb0085ff07008f87e90000000600f6
:1040b000889fbe008a9fbe00e00f5000e08f58002e
:1040c000e00f5900e08f59000c003d006044b8003b
:1040d0006055b8000000540081805c0002015d0062
:1040e00083815d00180020001500070008003d00d6
:1040f000180007000004eb00050037000004eb0087
:104100000f00070002003d00120007001800200009
:10411000dcff0700e00f5400060032006022b80008
:104120006033b8000000520081805a0002015b0039
:1041300083815b004f05be004f04be0000000600f7
:10414000e00f5200e08f5a00e00f5b00e08f5b0051
:10415000000006006044b8006055b8000402540036
:1041600085825c0006035d0087835d000000060019
:10417000889fbe008a9fbe008c1f7800e00f500011
:10418000e08f5800e00f5900e08f59000d003d000e
:104190006044b8006055b8000000540081805c00a5
:1041a00002015d0083815d001c0020000820e10009
:1041b00009a8e1000ab0e1000bb8e1000d003d00e4
:1041c000080037000006eb00e00f5200e08f5a00b5
:1041d000e00f5b00e08f5b0006003d006044b8002c
:1041e0006055b8000402540085825c0006035d003f
:1041f00087835d00aaff0700e00f5600060032002b
:104200006022b8006033b8000000520081805a007c
:1042100002015b0083815b004f0678004f05be0002
:084220004f04be00000006007f
:020000040000fa
:1042280048490000443a0000204d0000656d000038
:104238006f72000079200000666f00007220000095
:1042480052650000706f0000727400002044000086
:10425800657300006372000069700000746f0000ed
:10426800723a0000200000000d0a0000004800001b
:10427800494400002d4800004f530000543a000004
:10428800202e00002e2e0000203200006e64000058
:10429800205000006172000073650000200a0000d1
:1042a800000d00000a2000003d3d00003d3d0000db
:1042b8003d3d00003d3d00003d3d00003d3d00000e
:1042c8003d3d00003d3d00003d3d00003d3d0000fe
:1042d8003d3d00003d20000052650000706f000069
:1042e80072740000204400006573000063720000cf
:1042f80069700000746f00007220000044750000af
:104308006d700000203d00003d3d00003d3d000077
:104318003d3d00003d3d00003d3d00003d3d0000ad
:104328003d3d00003d3d00003d3d00003d3d00009d
:104338003d3d0000200a00000a0000000d0a0000b0
:10434800436f00006c6c0000656300007469000036
:104358006f6e0000733a000020200000000d00007e
:104368000a4d000061780000204e000065730000cf
:10437800746900006e6700003a2000002000000009
:104388000d0a000052650000706f00007274000092
:10439800733a000020200000000d00000a520000bf
:1043a800657000006f7200007449000074650000b9
:1043b8006d7300003a200000200000000d0a000084
:1043c80055730000616700006549000074650000ce
:1043d8006d7300003a20000020200000000a000051
:1043e8000d2d00002d2d00002d2d00002d2d00007d
:1043f8002d2d00002d2d00002d2d00002d2d00004d
:104408002d2d00002d2d00002d2d00002d2d00003c
:104418002d0a0000000d00000a4300006f6c000028
:104428006c65000063740000696f00006e20000076
:104438002020000020200000203a0000200000007a
:104448000d0a000020200000202000004461000028
:1044580074610000202000002020000020200000bf
:104468002020000020200000202000003a2000002a
:10447800000d00000a200000202000002055000048
:10448800736100006765000020500000616700004c
:10449800652000002020000020200000203a0000b5
:1044a800200000000d0a000020200000202000004d
:1044b800317300007420000055730000616700002c
:1044c8006520000049740000656d00002020000090
:1044d8003a200000000d00000a2000002020000003
:1044e800202300002055000073610000676500006c
:1044f80020490000746500006d7300002020000052
:10450800203a0000200000000d0a000020200000d2
:104518002020000031730000742000005265000064
:10452800706f00007274000020490000746500007c
:104538006d2000003a200000000d00000a20000055
:104548002020000020230000205200006570000099
:104558006f7200007420000049740000656d00004f
:1045680073200000203a0000200000000d0a00001f
:10457800202000002020000050610000726500002b
:104588006e74000020200000202000002020000081
:1045980020200000202000003a200000000d00002c
:1045a8000a20000020200000203100007374000061
:1045b80020430000686900006c64000020200000af
:1045c8002020000020200000203a000020000000e9
:1045d8000d0a000020200000202000004e65000089
:1045e8007874000020530000696200006c690000c4
:1045f8006e67000020200000202000003a20000004
:10460800000a00002d2d00002d2d00002d2d00008a
:104618002d2d00002d2d00002d2d00002d2d00002a
:104628002d2d00002d2d00002d2d00002d2d00001a
:104638002d2d00000a0000000d0a00005265000040
:10464800706f00007274000020200000203a000003
:10465800200000000d0a000052650000706f000085
:104668007274000049440000203a00002000000055
:104678000d0a0000496e00006269000074730000b2
:1046880020200000203a0000200000000d0a000051
:104698004f75000074620000697400007320000008
:1046a800203a0000200000000d0a000046650000c6
:1046b800617400006269000074730000203a000011
:1046c800200000000d0a000052650000706f000015
:1046d8007274000049740000656d0000202000001d
:1046e8003a200000000d00000a520000657000002a
:1046f8006f7200007454000079700000652000009b
:10470800203a0000200000000d0a00005374000049
:1047180061720000742000004269000074200000eb
:10472800202000003a200000000d00000a4200008e
:104738006974000073200000202000002020000081
:1047480020200000203a0000200000000d0a000090
:1047580050610000726500006e74000020200000a7
:1047680020200000202000003a200000000d00005a
:104778000a44000061740000614d00006f6400008d
:104788006573000020200000203a0000200000008f
:104798000d0a0000317300007420000055730000fa
:1047a8006167000065200000202000003a2000001a
:1047b800000d00000a5500007361000067650000e5
:1047c80020490000746500006d730000203a000065
:1047d800200000000d0a000020200000202000001a
:1047e80020200000476c00006f620000616c000030
:1047f8007320000020200000000d00000a75000052
:104808007361000067650000506100006765000083
:1048180020200000203a0000200000000d0a0000bf
:1048280072650000706f0000727400007369000008
:104838007a65000020200000203a000020000000d7
:104848000d0a000072650000706f000072740000ad
:104858004944000020200000203a00002000000009
:104868000d0a000072650000706f0000727400008d
:10487800436f0000756e00007420000020200000c7
:104888003a200000000d00000a5500007361000086
:104898006765000049740000656d00002020000075
:1048a8003a200000000d00000a5500007361000066
:1048b8006765000073200000202000002020000011
:1048c8004d6900006e6900006d7500006d200000e4
:1048d8002020000020200000204d0000617800000a
:1048e800696d0000756d000020200000200a00009e
:1048f8000d0000000909000000090000000d00007b
:104908000a55000073610000676500003a20000046
:104918000000000048490000443a0000204400001c
:104928006574000061630000680d00000a00000063
:1049380048490000443a0000205500006e6b000012
:104948006e6f0000776e000020640000657600003e
:1049580069630000650d00000a0000004849000076
:10496800443a0000204700006f7400002052000005
:10497800657000006f72000074200000446500003c
:104988007363000072690000707400006f720000a9
:104998000d0a0000000d00000a480000494400000c
:1049a80020450000727200006f7200002052000063
:1049b800657000006f7200007465000064200000dc
:1049c8003a200000200000000d0a0000000d000041
:1049d8000a480000494400003a20000053650000de
:1049e8006e640000696e00006720000052650000d8
:1049f800706f0000727400002044000065730000ae
:104a08006372000069700000746f0000722000007b
:104a180050610000727300006564000020650000aa
:104a2800766500006e7400000d0a00000048000062
:104a3800494400003a20000045720000726f0000ef
:104a4800722000007061000072730000696e00003f
:104a5800672000006465000073630000726900004d
:104a6800707400006f7200000d0a0000004800001a
:104a7800494400003a2000004f75000074200000ef
:104a88006f660000206d0000656d00006f72000009
:104a9800790d00000a00000048490000443a00006f
:104aa80020450000727200006f720000206700004d
:104ab80065740000746900006e67000020640000df
:104ac800657300006372000069700000746f000075
:104ad800720d00000a00000048490000443a000036
:104ae80020500000726f0000626c0000656d0000cd
:104af800206300006f6c00006c65000063740000a8
:104b0800696e00006720000072650000706f000089
:104b1800727400002064000061740000610d0000e0
:104b28000a00000048490000443a000020500000f4
:104b3800726f00006365000065640000696e000024
:104b480067200000746f000020720000756e00007e
:104b58002073000074610000746500000d0a0000f5
:104b680000480000494400003a2000005772000045
:104b7800697400006520000045760000656e00003d
:104b8800740d00000a00000048490000443a000083
:104b98002052000065730000657400002045000085
:104ba800766500006e7400000d0a00000000000029
:104bb8004445000056490000434500005f4e000090
:104bc8004f5400005f4300004f4e00004e45000068
:104bd80043540000454400000d0a00000041000055
:104be8007474000061630000682000006d6f0000ad
:104bf80075730000650d00000a000000766900006a
:104c0800643d0000002c00002000000070690000d6
:104c1800643d0000000d00000a0000005479000007
:104c2800706500005573000062440000657600005e
:104c380069630000653d0000004e0000756d0000ce
:104c48004f66000052650000706f0000727400002b
:104c580049740000656d00003d00000044650000d7
:104c680076690000636500003d4d00006f75000027
:104c7800736500000d0a000000440000657600001e
:104c880069630000653d0000506f0000696e000018
:104c980074650000720d00000a00000072650000d3
:104ca800706f00007274000049740000656d0000a8
:104cb8002d3e0000676c00006f620000616c000010
:104cc800732e0000757300006167000065500000d6
:104cd80061670000653d0000002000002020000002
:104ce80020680000696400005573000061670000d7
:104cf80065490000746500006d2d00003e750000d8
:104d080073610000676500003d0000004465000015
:104d180076690000636500003d4a00006f79000075
:104d280073740000696300006b0d00000a00000046
:104d38004465000076690000636500003d47000097
:104d4800616d00006520000050610000640d0000e6
:104d58000a0000006465000074610000696c0000ce
:104d6800732e000072650000706f000072740000fe
:104d78004c6500006e670000746800003d25000067
:104d880030340000780d00000a0000007044000074
:104d980065760000696300006552000070740000c9
:104da800696e0000666f00002d3e0000726500000d
:104db800706f000072740000733d00000000000076
:104dc8004a650000737400002077000061720000db
:104dd800746f0000736300000d0a0000000d0000ee
:104de8000a52000079730000205500005342000069
:104df800206600006f720000204100006d6900000d
:104e080067610000204300006f6d000070750000ae
:104e180074650000727300000d0a0000286300002a
:104e2800293200003032000031200000372d000008
:104e380062690000742c00002041000072740000b8
:104e4800757200002047000061640000617700006f
:104e5800736b0000690d00000a760000302e000018
:104e680031340000206200006574000061200000f9
:104e7800310d00000a00000030310000323300001c
:104e88003435000036370000383900004142000050
:084e9800434400004546000000
:020000040000fa
:104ea000705180004600de00614060000000060096
:104eb00004f02000a65080008602620010c3b300f8
:104ec000e08f52001e003200a550800005036200f2
:104ed00005402000850f530007003a00a4508000d1
:104ee000040fb2000040e900f00f520014003a0035
:104ef0006a40400000000600a650800006026200e2
:104f000005502000850f520002003a0022cabf005f
:104f100000000600a550800040c3b300041020002c
:104f2000848f520006003600a550800000c0e900c2
:104f3000f43f2000848f52000100360000c0e800da
:104f4000000006008042780060c0b30014a2200078
:104f50001442780084cf520008003a0004f0200088
:104f6000a55080000502620030c0b300e00f52007f
:104f700002003200142aef000040eb00000006009f
:104f80008042780060c0b30014a220001442780070
:104f900084cf520007003a00a550800030c0b30013
:104fa00004412000848f520002003a00142aec00d1
:104fb0000040eb00000006008042780060c0b300b3
:104fc00014a220001442780084cf520009003a0055
:104fd000a550800030c0b30004402000848f5200f0
:104fe00004003a009404a90070024200a450880012
:104ff0000040eb0000000600b450800094029000d6
:105000000560a10015029800940290000550a100cf
:1050100015029800684aed0068eab7000300320004
:1050200000ff2f00142ab60000000600694aed00b8
:1050300069eab7000411200003003a0070c0b30011
:1050400022eab70004502000a450880000000600a7
:105050000a00fa00889fbe008a9fbe008c9fbe0097
:10506000804478000144780082467800dc53800058
:105070002b0020000005eb004352dd0066034200d8
:10508000459e200065037b008603d100e1c36300d9
:10509000e1cf53003b003a004533de00614363003b
:1050a00003003a00e5427a0089cf520035003a0009
:1050b00066034200459e200065037b004433de000a
:1050c0006143630004003a000482420014429000ed
:1050d000884f52002b003a00c352dd006683420025
:1050e000449e200064037b004333de006143630081
:1050f00004003a008582e80064c27a008d4f5200b5
:1051000020003a000c4a90000482fb009c4a900068
:10511000c82add0084827200d5b79f00ac4a900097
:105120008582fb003c4a90004822dd0005027200a7
:10513000e4b79f00e9ef9f00f8ef9f008df79f0015
:105140008400200005002000768157009107200090
:1051500000c0eb0093bf9f00051f07009fb9970099
:10516000e04f500007003a004355dd00849e2000c8
:10517000040545001a4590008a49780010c0b30024
:10518000040037000a05e8008b05e900baff3a0081
:105190000b4078004f06be004f05be004f04be0016
:1051a0000080fa00000006000800fa00889fbe0098
:1051b0008a9fbe00d95380002ecaa9002eeaa900fa
:1051c0002b0020000005eb00489e20004352dd002c
:1051d000e6024200e8827a000503d10061436300e1
:1051e0000f00320068437a00c9429000854f530097
:1051f0004f003a008402440015439000d9429000c9
:10520000854f53004a003a000482e800e8427a00e1
:105210006942900084cf520045003a0043003700b5
:10522000894b90008783fb00194b90004833dd00c9
:1052300007037300e8037a00868f530019003a00d1
:105240008483e800294890000080fb00394b9000df
:105250004833dd0000037300e8837b00868f530032
:1052600010003a00472bde0061436300e14f53001a
:105270000b003a002eeaa800640242000403440036
:105280001640900024eab700c22ade00e1c26200a4
:105290000400320068407a001eeab70001003700bf
:1052a0002ecaa8004352dd00e8027a00e18f4200d6
:1052b0001f003a008482e80068807a00e10f400015
:1052c0001b003a00094b90000683fb00994b9000ad
:1052d000c83bdd008683730087bf9f00a94b900009
:1052e0008783fb00394b90004833dd0007037300d0
:1052f00096bf9f0068437a00c6f79f0004024400ef
:1053000014429000d4f79f00e8c27a00e5f79f00ae
:1053100084002000050020007081570091072000c4
:10532000931e0700e04f500001003a002ecaa8006b
:105330002ecaab000f0032004355dd00e4024500e9
:10534000449e2000050342001640900023eab70067
:105350006605450064037d004233de00614363005f
:105360001bc0b3000600320064c07a001eeab7001a
:10537000030037000a05e8008b05e90093ff3a00b7
:105380000b4078004f05be004f04be000080fa00bd
:105390000000060080427800e0cf520002003a0090
:1053a0006051800000000600545180000c0037005e
:1053b00024039000e00f5300080032002600900004
:1053c00004003700205b9000854f53000700320037
:1053d00010007800e00f5000faff3a001402780045
:1053e000e00f5200f2ff3a000400780000000600cf
:1053f0000200fa00881f78000204780014a220003e
:1054000014427800844f50000500320064c0b3009d
:10541000044c78008009eb00b311780022003700bb
:1054200001407800e3bf9f00daff0700efb9970063
:10543000e00f50001a00320090029000c92ade00ee
:10544000e1c26200100290000410b20005003200b8
:10545000004ceb00000b9000900b90008689be0082
:105460000d003700100290000402b200020032006a
:1054700014c1b30007003700100290000404b2000a
:105480000300320040589000004c780002003700c2
:1054900094c1b300044c7800054078000300370045
:1054a00044c1b300044c780010c0b3004f0478002e
:1054b0000080fa000000060014a2200014427800c8
:1054c000844f50000a003a0001407800b1ff070005
:1054d000e00f500006003200100290000470a0009f
:1054e00014009800100290000490a000140098008e
:1054f000000006000200fa00881f780000427800d1
:105500000204780065c0b30016a22000164378009c
:10551000864f52000f003a0001407800e3bf9f0021
:105520009cff070045c1b300efb99700e00f5000a2
:1055300008003200610464004d44dd001002900058
:1055400004d0a10008027200140098000310980013
:105550008042eb00054078004f0478000080fa009c
:1055600000000600004278000140780065c0b300ea
:1055700016a2200016437800864f52000b003a0016
:1055800084ff070045c1b300e00f50000700320060
:10559000100290000450a100140098001002900026
:1055a0000460a100140098008042eb0005407800e0
:1055b00000000600645180008083fb00d40a900044
:1055c000c82ade00e3826200878f520003003a009f
:1055d000940290000520b200210032001b6aef0007
:1055e00055518000e08f520026003a0005027800f5
:1055f00028003700e00f52001f003200540b9000cb
:105600004833de0063036300870f530017003a003e
:10561000e04f500003003200e34f500013003a0007
:1056200003003700140390000620b2000a00370080
:10563000140390000620b2000600320034039000ec
:10564000e00f530009003a0024039000360298004e
:105650000600370034039000e00f530003003a00c7
:10566000b450880015c0b3000c0037001402780055
:10567000e00f520007003a0095027800e08f5200d8
:105680000600320025029000e00f520001003200b7
:1056900024029000e08f5200d6ff3a0005407800c7
:1056a00000000600889fbe008a1f7800180037009f
:1056b00014047800100037009404780005003700c7
:1056c0001005780000f60700545180001402900085
:1056d0002a02980054518000140290002400900087
:1056e000e00f5000f6ff3a0004007800f6f50700de
:1056f000545180001902980050518000100290000f
:10570000e00f5200ecff3a00eff507005851880017
:1057100054518000e00f5200e5ff3a002c0af800d7
:10572000160af9004f0578004f04be00000006007d
:10573000889fbe000700370098049000180078008a
:10574000e1f50700405180000008eb00def507009e
:105750004951880048518000e00f5400f6ff3a009c
:10576000d0538000e00f500002003200d6f5070051
:10577000d853880080518000e00f500002003200b2
:10578000d1f50700302aef00c6ff07004f04be0026
:1057900000000600881f780068518000e00f540068
:1057a00007003a002002200039f507006051880008
:1057b000e00f50000f0032000808780001003700a9
:1057c000dbff07002c0af800160af900142aef0084
:1057d00010aaef00206aef00216aef006a0aa80011
:1057e0004400200094518800a4518800362aef001c
:1057f00010c0b3004f047800000006009002900033
:105800000550a10015009800900290000560a100cd
:1058100015009800900290000570a10015009800f6
:10582000900290000580a1001500980010039000e0
:1058300005fe2f008502630015009800900290007d
:1058400005c0a10015009800330898006033b80027
:1058500006089800170898000500200054009800da
:10586000650098000002eb00740898002108980079
:105870007200980004c2b30004589800100290000f
:105880000490a1001400980000000600900290000f
:105890000550a10015009800900290000560a1003d
:1058a00015009800900290000570a1001500980066
:1058b000900290000580a100150098001003900050
:1058c00005fe2f00850263001500980090029000ed
:1058d00005c0a10015009800330898006033b80097
:1058e00006089800170898006123b8005600980031
:1058f000670098008002eb00750898002108980066
:1059000072009800850f520002003a0004c1b300f3
:105910000100370004c3b30004589800100290003f
:105920000490a100140098000000060010029000ee
:105930000470a10014009800100290000480a100df
:10594000140098009002900004fe2f000482620070
:10595000140098001002900004c0a10014009800e8
:10596000310898006022b8000408980015089800d3
:105970000300200052009800630098008002eb00b2
:1059800075089800500a90000430b20006302000dc
:10599000860f520002003a0004c4b300080037002a
:1059a00006102000860f520004003a0004c6b3001f
:1059b00004589800954098000200370004c8b300ce
:1059c00004589800100290000490a1001400980060
:1059d000000006000400fa00889fbe000043780023
:1059e000020478000401be0064c0b30015a22000c8
:1059f00095427800854f530026003a0006f02000bb
:105a0000a45080000403630014c0b30005402000cc
:105a1000850f53001f003a0001407800c2bf9f006d
:105a2000d3bf9f005bfe070044c1b3004fb997008e
:105a3000e00f500017003200d00a90000530b2008d
:105a400084c1b30013003200a05a900054c1b300c7
:105a5000e0cf52000f003d00900290000502b2001e
:105a600014c1b3000b003a00900490000904b20086
:105a700024c1b30007003a00900290000520b20054
:105a800004c1b3000300320088007800a7ff0700bc
:105a900009427800044078004f04be000080fa00fc
:105aa00000000600100290000470a100140098008d
:105ab000100290000480a100140098009002900051
:105ac00004fe2f000482620014009800100290006f
:105ad00004c0a10014009800310898006022b800aa
:105ae0000408980015089800030020005200980050
:105af000630098008002eb0075089800500a90003f
:105b00000430b20006302000860f520002003a0036
:105b100004c5b3000800370006102000860f5200ad
:105b200004003a0004c7b300045898009540980058
:105b30000200370004c9b300045898001002900016
:105b40000490a10014009800000006000400fa0070
:105b5000889fbe0000437800020478000401be0064
:105b600064c0b30015a2200095427800854f530011
:105b700026003a0006f02000a450800004036300d1
:105b800014c0b30005402000850f53001f003a00e9
:105b900001407800c2bf9f00d3bf9f00fdfd0700fa
:105ba00044c1b3004fb99700e00f50001700320016
:105bb000d00a90000530b20084c1b3001300320057
:105bc000a05a900054c1b300e0cf52000f0035003e
:105bd000900290000502b20014c1b3000b003a001d
:105be000900490000904b20024c1b30007003a00f9
:105bf000900290000520b20004c1b30003003200ff
:105c000088007800a7ff0700094278000440780068
:105c10004f04be000080fa00000006000200fa00f7
:105c2000889fbe008a9fbe008c9fbe000045780002
:105c3000010478008204780024072000840f5400b7
:105c400003003200f4ff2700840f540009003a00db
:105c500019489000e14f400026003200a2c0b30076
:105c60000440bc000280e800a49d2000640378008a
:105c70001b0037005b518000611eb8000e0037002a
:105c80007b409000a2c0b3000440bc000281e80049
:105c9000a49d2000640379000c02be000901780075
:105ca000880078000a40780093bf9f00060001003a
:105cb0009b0578009fb99700e08f5500f0ff3a00f0
:105cc0002eeaab000b00320024cabf00a2c0b30012
:105cd0000440bc000281e800a49d20006403790018
:105ce000611ab80009017800880078000a4078003d
:105cf000060001004f06be004f05be004f04be0067
:105d00000080fa00000006000200fa008824ef007c
:105d100021cabf000f0032000042eb00e4ff9f00e9
:105d200064a2200014427800f4ff9f0024002000a9
:105d3000050020000f81e900a10620000c1c0700cf
:105d40001300200012a220001107200021cabf006a
:105d5000b2ff07006000b8008efe07000080fa0066
:105d600000000600881f78000244780034c0b300a9
:105d7000e1cf40000d003a00e04f54000b003a0024
:105d800085062000850f500003003a00deff070063
:105d90006a0aa90004003700b5062000850f5000ec
:105da00002003a006a0aa80008427800044078001d
:105db0004f04780000000600889fbe008a9fbe0046
:105dc0008c9fbe0000457800810478008205780031
:105dd00058518000611eb8000e00370078409000d6
:105de000a2c0b3000440bc0064014100a49d200097
:105df00064037900e00f5300050032000c02be007e
:105e00000b017800890078000a4078000600010044
:105e100018047800e00f5400f0ff3a004f06be006f
:105e20004f05be004f04be0000000600f287470089
:105e3000889fbe008a9fbe008c9fbe008e1f780088
:105e4000585180002e2aa9002e4aa800c453800071
:105e5000b44478000402e800344078008082fb00fb
:105e6000b44078000183fb004833dd0005034300a4
:105e7000d6b79f000402e800b4427800e5e79f002f
:105e80002442900084ef9f00c4e79f000045eb0090
:105e90007e8157000a697800240020000500200058
:105ea0009106200000c0eb00b11b07008a4f500094
:105eb00003003a0080c2b30022eab7001ac0b30060
:105ec0008984fb0009007800780ab4008045eb0063
:105ed000b300370005007800304678003042780083
:105ee000e94f52000c003a002e2aa8001042780018
:105ef000044078001feab70062026200040032002a
:105f00002e6aab00020032002e4aa90017003700ab
:105f10002e6aa90015003700e44f520013003a0022
:105f20001047780000027800d4467800d44078000a
:105f3000f1e79f0054407800d44078005441780045
:105f4000e4b79f002ecaab000400320034a2200048
:105f500014427800a4e79f0009003700fe81570033
:105f60003bfc0700e04f500005003a000c86fb00a8
:105f70008c84440009007800780ab4008a00370055
:105f8000080278000100370014027800e00f520088
:105f900004003200e44290008ecf5200faff3a0033
:105fa0000d0037008000200039f307000002780060
:105fb000e00f52000f0032006e429800afe09700f1
:105fc000714298008002eb001502980025029800ab
:105fd000080a7800040478006000200084bf9f0055
:105fe0002bf30700000778000fba9700e00f570067
:105ff0009a003a006fb297000400e8005f00370093
:106000002e0298000c86fb008c844400cc53800048
:10601000090046008045eb000002eb008802780092
:106020000a4478004d00370010457800800678005b
:1060300056c0b300dd4f1300040032000a85fb0098
:106040008a844400090046004400370020022000f2
:1060500084bf9f00f5b79f000df307000003780091
:10606000dd437800275b98005d407800305b980046
:10607000dd4078008183fb0047039800dd40780015
:106080000180fb004800dd008703400047039800c3
:106090009d4390008783fb00270398000fba970069
:1060a000140398001600900000a0a00010039800b0
:1060b000160090000090a000100398006000b80047
:1060c000000b9800110b9800045b98002fe09700dc
:1060d000105b9800560890000030b200ffb29700a5
:1060e00001102000810f500011003a00e08f530092
:1060f00002003a001700200027039800a603900032
:10610000f08f53000200360007012000270398009b
:10611000a60390008703e900100020008703dd003c
:10612000270398009603900007a0a100170398008a
:10613000a6039000370398002e009000000b780013
:10614000260798008b45e8000a85fb008a844400f6
:1061500009004600e00f530007003200dfb097004f
:10616000818f5400070031007fe3970086cf5500f0
:10617000adff390003003700050478001ac0b300f2
:10618000020037000845780005047800ffe3970017
:1061900087cf5500020032001ac0b3000600370056
:1061a000e04f550004003a00800278005fb097008d
:1061b000808f540047ff3900e00f54001600320072
:1061c000e04f550018003200130037001805780022
:1061d0000b00370099007800110498000300370085
:1061e00010027800a404980037f3070029009000fb
:1061f000e00f5000faff3a000900780032f3070080
:1062000098049000e08f5400f2ff3a0008007800f4
:106210002df307000a047800e00f5400ebff3a006a
:1062200008407800070037006fe097001eeab700cb
:106230008fe897000182fb00345188005851880094
:1062400010c0b3004f0778004f06be004f05be00d8
:106250004f04be002f01b100000006009402900020
:10626000050f78002d4798008002eb002507980065
:106270001e029800e0cf560061ff320061ff370038
:106280000200fa00889fbe008a1f7800f8ff2700ee
:106290001d003700a451800082a32000e20f5200ad
:1062a00004003c000401e8006c11b90085a3200043
:1062b000050141009200780024072000848f5000df
:1062c00002003200888f500004003a000281e8008a
:1062d000a300200021cabf0050fe070065248000f3
:1062e0008c24ef00362aed00a4518000e20f52000a
:1062f00003003c000402e800a451880001003700bc
:10630000342aef0065248800b4518000e00f520069
:10631000e0ff3a0084508000e10f420003003200a9
:10632000100af800140af90010aaef0008f0200083
:10633000a05080008002640004202000848f52005e
:106340003b01320006003e00e08f52000e0032009a
:1063500004102000848f520011033a0076003700a9
:1063600004402000848f5200c30232000410b000a9
:10637000848f5200da02320004302000848f5200f1
:1063800007033a0059013700a8508000080fb200f7
:10639000f00f54004500320004022000840f540026
:1063a00047003200e00f5400fd023a0056fe07009d
:1063b00064518000080a7800180298009402900046
:1063c00005a0a00015029800940290000590a0007e
:1063d000150298009402900005d0a00015029800c4
:1063e0004501200005129800050420004502980090
:1063f0006033b800060a9800170a9800285a9800d7
:10640000085a9800d40a90000580a1000590a100c8
:10641000550a980080c2eb00155a980030c0b300ae
:1064200069eab700084078001eeab7001feab70023
:1064300020eab7007851880058518800c850880079
:1064400068248800f40f200054248800c00820002d
:106450008224b600d50720000524880088248800ff
:106460007424880004a020004822de00c424880090
:1064700084002000a4248800a5002000a524880012
:10648000a424880004032000342488002400200071
:106490003425880048258800b8248800aae4a9008b
:1064a000a404200004258800b8023700a4a6200018
:1064b0001442780061426200b9023200fa013700ea
:1064c00085ff9f0024c3b30094ff9f002400200099
:1064d00005002000688157009106200000c0eb00f5
:1064e000231a0700e04f5000100032001400200073
:1064f000442488008ec0a900740680000480a10096
:106500000490a00004a0a000740688009ec0a8000b
:1065100004ff2000a55080000502620070024200c6
:10652000a45088008cc4a8009d0237006a0aa90004
:106530000401200099023700a4508000040fb2002b
:1065400006022000860f52005700320005003e0070
:10655000e00f52000a003200f00f520090023a00a1
:106560001200370006032000860f52008700320019
:1065700005042000850f520089023a00a800370068
:10658000a45080006f02620003003200e20f52004c
:1065900083023a00c401370014002000542488000c
:1065a0008c04a800b40f200045023700a4508000de
:1065b0006f026200e20f520034003200e40f52001a
:1065c00034003200e00f520075023a008051800022
:1065d000e00f5000010032003bf207008000200075
:1065e000abf1070080518800e00f50001501320028
:1065f0001e6aef001f6aef002e2aef0030c0b300c2
:1066000068eab700d400200054258800ac24ef00cd
:10661000ae24ef00b024ef00b224ef00b424ef006a
:10662000b624ef00b824ef00ba24ef00bc24ef003a
:10663000be24ef00c024ef00c224ef00c424ef000a
:10664000c624ef00c824ef0094e4ab0006003a0033
:106650002e0aa80000c8b30020eab70004082000f2
:10666000b4248800aae4a8009424a8009424a900d3
:106670002e8aa9002eaaa9009484a8003403200021
:10668000945088006d0242000f0237009484a900e4
:1066900009023700f400200064248800f40f200071
:1066a0008424880039023700a45080006f02620001
:1066b000e10f52001300320003003900e20f5200d4
:1066c00037023a001c003700d0538000e00f500022
:1066d00002003200fcf107007a2aef0083518000ab
:1066e00004c8b3008449780064c0b30094419800a2
:1066f0000042eb00a441980015c0b300b5419800da
:10670000b300370066518000160290000420b200ea
:106710002302320016029000850262008b013200d3
:106720008451800044429000e94f5200e8013a0051
:1067300054c3b300cc013700885180001842780060
:106740000480fb0052f10700d0538800e00f500096
:10675000bc00320018487800f84290008582fb00a7
:10676000645180004502980008007800d6f10700c7
:10677000645180004400900045f10700805188007a
:10678000e00f5000c1003a00ae003700a450800076
:106790006f026200e10f520019003200030039005d
:1067a000e20f5200fe013a00b8003700188aab0031
:1067b000fb013a008151800004c8b300844878008e
:1067c00064c0b300944098000042eb00a4409800dd
:1067d00015c0b300b5409800c4409800d44098005c
:1067e000d553800095427800e5409800f440980029
:1067f000d3538000134078000082fb00c9003700ab
:1068000066518000160290000420b200e4013200bc
:106810001602900085026200ad013a004b0137007c
:1068200061fa0700a0508000000464002c003700cb
:10683000a4508000040fb200d9013a00a650800095
:106840006f036300e10f53001300320003003900af
:10685000e20f5300d2013a001500370010c0b30018
:1068600021eab700815180008448780055c0b30008
:106870009540980015a2200095427800a540980008
:10688000b4409800c4409800d4409800e440980078
:10689000f4409800210137006451800014039000f7
:1068a00085026300be01320014029000250137000a
:1068b00074518000610262004722dd0015a22000b1
:1068c0009542780004c272000440780020eab700c4
:1068d00030c0b30068eab700a4508000040464002c
:1068e0000810b000a8508800ad013700a450800007
:1068f000040fb20005022000850f5200660032002e
:1069000005003e00e00f52000d003200f00f520073
:10691000a3013a001c00370005042000850f520037
:10692000d7003200f0824200850f5200e2003200b0
:1069300005032000850f520099013a0084003700ba
:10694000d453800014549000084078006beab700dc
:106950000700370094049000140078005af10700f3
:10696000405180000008eb0057f1070049518800b2
:1069700044518000e00f5200f6ff3a00e04f54000f
:1069800082013a0037013700a45080006f02620094
:10699000e10f5200e600320003003900e20f52001e
:1069a0007f013a00130037008351800004c8b30010
:1069b0008449780064c0b300944198006b4aed00ac
:1069c000a041980024c0b300b44198000042eb00fd
:1069d000c4419800d441980085c0b300e5419800b7
:1069e000f4419800840020000401780083007800be
:1069f0004d00370060002000a5f00700000478007b
:106a0000e00f54000f00320089518000638544007c
:106a10008984e8001a4278000480fb004800dd0009
:106a2000994278000582fb000400400098f00700be
:106a3000000c7800e00f500004003a0008007800d5
:106a400021f1070034c3b300070137001a4578006d
:106a50000a82fb004822dd00994478008982fb000d
:106a600005024200244098004822de00344098008d
:106a7000445180001404980048518800c053880095
:106a8000b5a62000954278004544980030c0b30078
:106a900068eab7003d013700a45080006f02620031
:106aa000e10f5200a200320003003900e20f520051
:106ab0003b013a001f0037008151800004c8b30039
:106ac0008448780064c0b300944098006b4aed009d
:106ad000a040980024c0b300b44098000042eb00ee
:106ae000c4409800d44098004451800014027800bb
:106af00024429000e4409800445180001402780041
:106b000034429000f4409800445180009401780091
:106b1000a34290008582fb00334290004822dd00b2
:106b200005027200820020006051800033fb0700e4
:106b3000e700370030c0b30068eab7006b4aed00e9
:106b40006beab7000431200014013a000f0137004e
:106b5000a45080006f02620005002000e30f520085
:106b6000e08f5a000e013e00046001000300370070
:106b70002e0037006e0037003a003700c9fa0700d0
:106b8000e5a1200095427800e0cf520010003a00c5
:106b9000280af8006c0af90009003700140278008e
:106ba000c4538800a1fc0700e04f500019003a00d0
:106bb000bcfa0700645380001402900064538800fc
:106bc00064538000e00f5200f4ff3a0011003700d8
:106bd0004451800064538800010037001402900083
:106be000e00f52000300320044439000854f5300f1
:106bf000faff3a006453880014027800c4538800f6
:106c00008afc0700e04f500002003a00a5fa070096
:106c10006c2aef002e4aab00ad00320064538000b6
:106c2000e00f5200aa003a001300370074518000b0
:106c300064026200d5003a002e4aa800815180000b
:106c40008448780034c0b300944098002e6aab00aa
:106c500001003a0044c0b300a44098000042eb0099
:106c60002800370030c0b30068eab70064538000e2
:106c7000e00f5200c5003a0044c3b3007a00370069
:106c800014a22000144278000482fb0005002000ba
:106c90000001eb00c107200000c0eb003418070022
:106ca000e04f5000be003a0004ff2000a0508000da
:106cb00000026200b8003700a45080006f0262003a
:106cc00005002000e30f5200e08f5a00b4003e00a0
:106cd0000460010003003700150037001d00370075
:106ce0001f003700815180000042eb00844878008b
:106cf00095c0b30095409800e5a12000954278002a
:106d0000a5409800b4409800c4409800d440980032
:106d1000e4409800f44098000002eb008401780001
:106d20008200200060518000d8fa07006800370018
:106d300065518000150290000420b20098003200d6
:106d4000150290000410b20061003a00aaf8070092
:106d50009300370030c0b30068eab7005c0037002a
:106d600004f02000a5508000050262000410b0006d
:106d7000a45088002ecaab001300320031a22000bc
:106d80009140780001407800a2c0b3000440bc00ec
:106d9000a49d200082024200640279003501900027
:106da000c501900021cabf0004000100e04f50005f
:106db0001c003a0090c3b30022eab7000450200040
:106dc000a450880017003700585180009ac3b300c0
:106dd0000950200011003700f84090000140780071
:106de000a2c0b3000440bc00a49d20008202420067
:106df0006402790035019000c501900021cabf00ee
:106e000004000100e04f500003003a000a407800ff
:106e100022eab700a950880018047800e00f540057
:106e2000edff3a002eeaab005d00320041a22000e7
:106e30009140780001407800a2c0b3000440bc003b
:106e4000a49d200082024200640279003501900076
:106e5000c501900021cabf0004000100e04f5000ae
:106e60004f003a0094c3b3000440780022eab70010
:106e70000450200049003700a4508000040fb200e5
:106e8000f00f520046003a00a45080006f026200ea
:106e9000e30f520007003200e50f52000e003200ef
:106ea000e10f52003e003a009444a8005401200033
:106eb000030037009444a9009404a800b400200003
:106ec00094508800040420000424880082c4a80090
:106ed000142aec0032003700a5508800300037003b
:106ee000a4508000040fb2002d003a00850020005d
:106ef000a524880064248800f50f2000552488000c
:106f0000c00820008224b600d6072000062488008e
:106f100084248800752488008c04a80024a2200002
:106f20001442780045c3b300c1c6b300854f520078
:106f30001000320006003e008140e800e74f52009a
:106f40000c00320081c0e8008542e90006003700ed
:106f500051c6b30055c3b300854f5200050032003f
:106f6000e9c04000e4c24200854f520001003200f7
:106f700001c7b3008180fb00140020000500200041
:106f800062a2200021cabf007917070004ff200079
:106f9000a55080000502620070024200a4508800e3
:106fa0004f0578004f04be000080fa000000060084
:106fb000e04f500013003a00555180000e0037009a
:106fc00015039000090037002602900004003700e6
:106fd0009403900007b0a1001702980014027800f3
:106fe000e00f5200faff3a0016037800e00f53005a
:106ff000f5ff3a0095027800e08f5200f0ff3a006a
:1070000000000600e3f80700e00f50000300320024
:107010001002900004b0a1001400980000000600c7
:107020000400fa00889fbe008a9fbe008c1f780073
:107030000144780082447800030578000406780053
:1070400005027800860178008745780065c0b300a6
:1070500016a2200016437800864f500050003a00d8
:1070600007f02000a55080008583630015c0b300a1
:1070700006402000868f530049003a006551800089
:10708000150390000620b20005c1b3004400320091
:10709000ebcf54001c003a0056518000010037002d
:1070a00016037800e00f53003c003200e6429000e7
:1070b0008582fb008c8f5200f9ff3a003e003700ba
:1070c000a702900004003700950390000720b2004b
:1070d0003200320095027800e08f5200faff3a0049
:1070e000960290000100370095027800e08f520070
:1070f0002a003200a54390008783fb008a8f53004b
:10710000f9ff3a0031003700e1cf54000a003a009d
:10711000e00f550008003a00e24f540006003e0020
:107120000c407800a3bf9f0094bf9f00a0ff070002
:107130001fba9700afb99700815180008848780046
:1071400099409800aa4098004855de00ba4098003f
:10715000cc4098004866de00dc409800e44098008f
:10716000c822de00f540980060518000afea970029
:1071700015589800e0cf550004003a008200200026
:10718000c2f907008b42780005003700820020001a
:107190009af907008042eb000100370035c0b300c8
:1071a000054078004f0678004f05be004f04be0032
:1071b0000080fa0000000600a603900035c0b3006e
:1071c000e08f5300beff3a00f5ff3700250398001b
:1071d000d9ff370075518000e1826200d4cdb30041
:1071e00001003a00d4c5b300b6508000d60a900022
:1071f0000530b20001003a000444a100d60a900014
:107200000530b20006102000868f520001003a00bf
:107210000404a1000482fb005425880004a220007d
:10722000144278000482fb00b42488008180fb00b3
:10723000c408dd00f007b20000807000f024880070
:10724000188aa80000000600e94f50000f003a001d
:10725000745180007002620045a0200001003a00d5
:1072600005a02000765180004433de000683ea004a
:10727000610363004433dd00745180000440a100c9
:107280000602720074518800230037007451800098
:107290000402b200c5a0200001003a00e4825200be
:1072a000765180004533de000683ea006103630007
:1072b0004533dd00745180000450a10006027200c5
:1072c00074518800ed4f500013003a00b450800014
:1072d0007400900004099000940990004403900009
:1072e00001002000020050008380580007002000a9
:1072f000860f5000878f580002003600440390002c
:107300002300370074009000040b9000940b900051
:10731000060350001e003700b4508000540b90004c
:107320000630b20007102000870f530005003a0016
:10733000e94f50000e003200040b9000940b9000b7
:107340003b00370054019000e401900004089000d5
:10735000940890004403900000005100818059007f
:1073600007002000860f5000878f5800020036006b
:10737000440390002e00370054009000e400900079
:10738000040b9000940b9000060350002800370077
:10739000240a90000d003700b40b9000340a9000ce
:1073a000144090000080fb000000e8006600b90077
:1073b000e70378009702980005003700b40b9000af
:1073c0000408900094089000008243009402980002
:1073d0000042eb0094429800f63fb20004c02f0038
:1073e0001502620006027200840a7800b75080001d
:1073f000170090004b00de00610060004e00dd00d1
:1074000004e0a10000027200840a78009703900053
:10741000ca3bde00e1836300cb3bdd0004b0a1008a
:107420000702720004f0a000840a78000000060041
:10743000d40b90000730b20000102000808f530062
:10744000deff3a00d4ff3700889fbe008a9fbe004f
:107450008c9fbe008e1f7800a4508000c950800011
:10746000f08464006a013a00ca508000610565003a
:10747000c5003a000a4078004ef80700e04f50007f
:10748000c0003200b8508000085a9000040fb200cb
:1074900005022000850f520022003200f0824200d7
:1074a000850f52003b003200f00f520051013a00ac
:1074b000085a90006f026200e10f5200090032008a
:1074c00003003c00e00f5200460032004901370043
:1074d000e20f520011003200ef0f520045013a0056
:1074e0007800370008089000980890005004980031
:1074f000610498001802900004b0a00014049800e1
:1075000090c0b30050ff07002858900091c0b3000e
:1075100030ff0700180aa8003d0137000a5c9800f8
:1075200044003700085a90006f026200cfa2de00cc
:10753000046001002b003700f1ff37000d00370019
:107540003a0037002b0137002a01370029013700a4
:1075500028013700270137002601370025013700b1
:1075600024013700230137002201370021013700b1
:1075700054003700080a9000980a900054049800bc
:10758000650498001802900004b0a000140498004c
:107590001c003700085a90006f026200cfa2de0084
:1075a000046001000f003700160037001a00370092
:1075b0001e0037000f0137000e0137000d013700a4
:1075c0000c0137000b0137000a01370009013700b1
:1075d00008013700070137000601370005013700b1
:1075e000380037001802900004b0a100140498007d
:1075f000d0c0b30014ff070028589000d1c0b300da
:10760000c3ff370010c0b3000fff070028589000d9
:1076100011c0b300beff3700080a9000980a90001e
:107620005404980065049800b2ff37000042eb0054
:10763000045c9800180290000490a00014049800c4
:10764000b4518000e30f52004b003c000402e800fc
:10765000b451880094518000e20f520003003c00b6
:107660000402e8009451880001003700322aef003c
:10767000955180006c2bb900060278002707200086
:1076800086a3200007337a000683e8000403430042
:107690000808900098089000008bbe008502e80062
:1076a0006c2bb90025a32000b808900081327b0024
:1076b000ee824200848242000043eb009642980032
:1076c000240037000042eb00045c98001802900090
:1076d0000490a00014049800b4518000e30f5200fd
:1076e00025003c000402e800b45188009451800059
:1076f000e20f520003003c000402e80094518800ad
:1077000001003700322aef00955180006c2bb90040
:1077100006027800f7ff270086a3200007337a00cf
:107720000683e80004034300000beb0036137800e7
:107730008502e8006c2bb90025a320008682420058
:10774000800aeb0005a4200084824200c858900003
:1077500091429800285b9000864a780025a420007a
:107760000482420038589000004a7800185c90006b
:10777000184298000200370084c0b300345c9800bf
:107780008044eb00180aa800182aab008e003200d3
:107790009f003700b8508000085a9000040fb200d4
:1077a00005042000850f520004003200f0824200e0
:1077b000850f52007a003a0012003700085a9000f4
:1077c0006f026200e10f520009003200ef0f520019
:1077d00046003200e00f520071003a0090c0b30042
:1077e00099fe07002858900091c0b300110037009f
:1077f0000042eb00045c9800a8009000310498005f
:1078000012003700085a90006f026200e10f520028
:107810000a003200ef0f520034003200e00f520035
:107820005f003a0010c0b30087fe070028589000a0
:1078300011c0b30067fe0700750037000042eb007f
:10784000045c98002802900034049800180290000c
:107850000490a00014049800b4518000e30f52007b
:107860004a003c000402e800b451880094518000b2
:10787000e20f520003003c000402e800945188002b
:1078800001003700322aef00955180006c2bb900bf
:10789000060278002607200086367a000403460098
:1078a0000808900098089000008bbe008502e80050
:1078b0006c2bb90025a32000b808900081327b0012
:1078c000848245000043eb0096429800285b9000bc
:1078d000864a78000402450038589000004a780033
:1078e000185c9000184298002a0037000042eb0014
:1078f000045c9800a80090003104980018029000e1
:107900000490a00014049800b4518000e30f5200ca
:107910001e003c000402e800b4518800945180002d
:10792000e20f520003003c000402e800945188007a
:1079300001003700322aef00955180006c2bb9000e
:10794000060278008e367a0004034600000beb0036
:10795000361378008502e8006c2bb90025a32000bf
:1079600086824200800aeb0084824500485b9000da
:107970009642980028589000804a780004024500fa
:10798000b8589000014a7800d5ff370084c0b30092
:10799000345c9800e0cf5400100032000100370042
:1079a00019c0b300b45080008042eb00055a980023
:1079b000a402900035029800940290000590a00067
:1079c00015029800050037008da320000d86e80001
:1079d000e60546000b85e800feff270030c0b30037
:1079e000f4f60700e04f50006aff3a00182aa8009a
:1079f000070037000042eb00045c9800180290007a
:107a00000490a0001404980019c0b3005dff370073
:107a10004f0778004f06be004f05be004f04be0062
:107a20000000060064518000140290000420b2009f
:107a300010c0b30014003200505180000e00370017
:107a40001002900009003700a402900004003700e3
:107a5000150390000620b2000a003200950278005b
:107a6000e08f5200faff3a0014027800e00f520053
:107a7000f5ff3a0010007800e00f5000f0ff3a00e8
:107a80000000060010c0b30000000600881f780048
:107a90000144780064c0b30015a22000954278002c
:107aa000854f500014003a0006f02000a0508000de
:107ab0000003630014c0b30005402000850f53008d
:107ac0000d003a00d7ff07000043780024c0b30040
:107ad000e04f530008003a00084078001eeab70063
:107ae00080c2eb0064518000155a980004332000d6
:107af000a450880006427800044078004f047800c3
:107b0000000006008ec0a90082c4ab001200320043
:107b100080c4ab001000320004042000042488005c
:107b200094508000e00f52000b003200122aed004a
:107b300094508000e00f520007003a0082c4a90070
:107b400004f02000a050800000026200e00f52000c
:107b500001003200142aec008cc4ab000b00320090
:107b60008ac4ab00090032008cc4a90004042000c0
:107b700054248800a550800070025200848f520067
:107b800002003a0004102000845088008c04ab00ee
:107b9000060032008a04ab0004003200140020000a
:107ba000542488008c04a900102aef008c64ab00d8
:107bb000c50032008a64ab00c30032008c24ab00e5
:107bc000080032008a24ab0006003200b450800066
:107bd000540a90000430b20005102000850f5200b6
:107be000b9003a00188aa900962480008400200079
:107bf00054248800b4508000a45a9000f7248000d8
:107c000085826b00ef826200ae003a00e8026300fa
:107c100064036300e08f52000200320085a0200060
:107c20000100370005a02000e00f530001003200e2
:107c3000e482420006c02300150363000780200091
:107c4000870f530029003a00f63f20001503630018
:107c5000040890009408900006004000e08048006e
:107c6000000a9800110a98008002eb00750a98003b
:107c700094039000cb3bde008783ea00e18363003e
:107c8000cb3bdd009402900005b0a100878272001a
:107c900015029800845a9000f0cf5200080032007c
:107ca000845b900005c2b30085cf5300040032000e
:107cb000845b9000f0c2420085cf530024003a005c
:107cc00004089000940890007403900007002000be
:107cd000860f5000878f58007a0039006033b80053
:107ce000060a9800170a98005300370007c02000c2
:107cf000870f53000300320007c02200870f530094
:107d000023003a00f63f20001503630004089000aa
:107d10009408900006004000e0804800000a9800a7
:107d2000110a98008002eb00750a980094039000f5
:107d3000cb3bde008783ea00e1836300cb3bdd00c1
:107d40009402900005b0a10087827200150298008d
:107d5000d40a90000530b20007102000878f52002f
:107d600032003200c4029000850f53002f0039000a
:107d7000040890009408900054039000e4039000dd
:107d8000860f5000878f58004e00390027003700bb
:107d900005802200850f53002a003a0094029000cb
:107da00005c0a00015029800f40a90008502e800c2
:107db000750a9800d40a9000c82ade00e3826200a7
:107dc000e28f520008003200e38f520003003200bd
:107dd000e18f520004003a0014003700a45a9000ca
:107de000e0cf52001100350014039000050022007e
:107df0008502630033003200740b900084129000ff
:107e0000850f53002f003600940290000560a000fb
:107e10001502980075c1b300455a9800845a900025
:107e2000f540b300055a98002600370094029000f0
:107e30000580a00015029800845a90008542e80051
:107e4000f8ff370005802300850f530005003a0036
:107e5000940290000550a0001502980015c1b300cf
:107e6000edff3700140390000643e8007f03630032
:107e70009403900005fe2f008582630086827200c5
:107e80001502980094029000ff826200f38f520066
:107e90000c003400940290000560a00015029800c8
:107ea00035c1b300455a9800845a9000f540b3009c
:107eb000055a9800f40f2000742488002400200044
:107ec0005424880060fd07008c44ab002900320078
:107ed0008a44ab002700320044002000542488006c
:107ee0005551800000302000071020001800370096
:107ef00025029000e00f520014003200240290008e
:107f000010003700540b90000630b200800f530071
:107f100002003200870f530006003a00340390003d
:107f2000e00f530003003200340390000603e90021
:107f3000360298001403900006c0a10016029800b3
:107f400014027800e00f5200eeff3a00950278002c
:107f5000e08f5200e6ff3a00180aa900182aa9008b
:107f6000184aa900186aa900054078001aeab70063
:107f700035fd07008c24ab003b0032008a24ab00a7
:107f800039003200188aa900b4508000d40a900049
:107f90000530b20006102000868f52002e003200fd
:107fa000140390000643e8007f03630094039000ed
:107fb00005fe2f00858263008682720015029800fc
:107fc00094029000ff826200f38f5200220034007e
:107fd0008ee4ab000200320005c2b300455a98009f
:107fe0008ea4ab000200320015c2b300455a9800bf
:107ff0008e84ab000200320025c2b300455a9800bf
:108000008e64ab000200320035c2b300455a9800be
:108010008e44ab000200320045c2b300455a9800be
:108020008e24ab000200320055c2b300455a9800be
:108030008e04ab000200320065c2b300455a9800be
:10804000940290000560a00015029800845a9000e8
:10805000f540b300055a9800f40f200074248800fe
:108060002400200054248800000006009440800072
:10807000e20f520002003a003400200094408800d1
:108080000000060005408000e80f500035003c006d
:1080900056458000610363004833dd000580a10080
:1080a0008682720064458000610262004922dd0020
:1080b0000590a1000482720075458000e182620093
:1080c000ca2add0004a0a100050272000440880055
:1080d0000168a9000188a90001a8a900b445800091
:1080e000610262004522dd00154080000550a100bc
:1080f00004827200c5458000e1826200c62add006c
:108100000460a10005027200144088004441800010
:10811000e00f520002003a000088a8000600370075
:108120000088a900f50f2000850f520002003a00d8
:1081300000a8a8000100370000a8a9005441800051
:10814000e00f520002003a0000c8a80047003700c4
:1081500000c8a900f50f2000850f52004100320031
:108160004200370026468000610363004833dd008b
:108170000580a100868272003446800061026200a0
:108180004922dd000590a10004827200154680009e
:10819000e1826200ca2add0004a0a100050272008b
:1081a000044088000168a9000188a90001a8a9006d
:1081b00054458000610262004522dd0015408000c8
:1081c0000550a1000482720085458000e1826200b2
:1081d000c62add000460a100050272001440880078
:1081e00044418000e00f520003003200c54580008a
:1081f000e18f520002003a000088a8000100370019
:108200000088a900f50f2000850f520003003200fe
:10821000a4458000e10f520002003a0000a8a80027
:108220000100370000a8a90054418000e00f52006f
:108230000300320095458000e18f520002003a00b1
:1082400000c8a8000100370000c8a900f50f2000f1
:10825000850f520003003200b4458000e10f520048
:1082600002003a0000e8a8000000060000e8a900ab
:1082700000000600a44f8000b54f8000f6e8200003
:10828000860f5200e08f5a0057003a00c44f80001a
:10829000d54f8000e30f5200e08f5a0052003a00a1
:1082a000f49f200014427800e04f520020003a0072
:1082b00074458000610262004822dd0005408000b4
:1082c0000580a1000482720087458000e18363007d
:1082d000c93bdd000490a100870372006645800061
:1082e000610363004a33dd0007a0a1000683730029
:1082f00055458000e1826200cb2add0006b0a10076
:108300008502730094458000610262004c22dd000a
:1083100005c0a10004827200a5458000e1826200d0
:10832000cd2add0004d0a1000502720004408800bf
:10833000d4458000610262004522dd0015408000c6
:108340000550a10004827200e5458000e1826200d0
:10835000c62add000460a1000502720014408800f6
:1083600045418000e08f52000300320064418000ec
:10837000e00f520002003a000088a8000100370018
:108380000088a900f40f2000848f520003003200ff
:1083900065418000848f520002003a0000a8a800c6
:1083a0000100370000a8a90055418000e08f52006d
:1083b0000300320074418000e00f520002003a00d6
:1083c00000c8a8000100370000c8a900f40f200071
:1083d000848f52009b00320075418000848f5200d0
:1083e0009a003a0097003700f49f2000144278006a
:1083f000e80f500044003c00e04f520020003a00db
:1084000064458000610262004822dd000540800072
:108410000580a1000482720057458000e18363005b
:10842000c93bdd000490a1008703720076458000ff
:10843000610363004a33dd0007a0a10006837300d7
:1084400085458000e1826200cb2add0006b0a100f4
:108450008502730094458000610262004c22dd00b9
:1084600005c0a10004827200a5458000e18262007f
:10847000cd2add0004d0a10005027200044088006e
:10848000b4458000610262004522dd001540800095
:108490000550a10004827200c5458000e18262009f
:1084a000c62add000460a1000502720014408800a5
:1084b00044418000e00f520002003a000088a8000a
:1084c000060037000088a900f50f2000850f520034
:1084d00002003a0000a8a8000100370000a8a90087
:1084e00054418000e00f520002003a0000c8a8008a
:1084f0005600370000c8a900f50f2000850f520074
:108500005000320051003700e04f520020003a0086
:1085100034468000610262004822dd000540800090
:108520000580a1000482720027468000e183630079
:10853000c93bdd000490a10087037200164680004d
:10854000610363004a33dd0007a0a10006837300c6
:1085500045468000e1826200cb2add0006b0a10022
:1085600085027300f4458000610262004c22dd0048
:1085700005c0a1000482720005468000e18262000d
:10858000cd2add0004d0a10005027200044088005d
:1085900054458000610262004522dd0015408000e4
:1085a0000550a1000482720085458000e1826200ce
:1085b000c62add000460a100050272001440880094
:1085c00044418000e00f520003003200c5458000a6
:1085d000e18f520002003a000088a8000100370035
:1085e0000088a900f50f2000850f5200030032001b
:1085f000a4458000e10f520002003a0000a8a80044
:108600000100370000a8a90054418000e00f52008b
:108610000300320095458000e18f520002003a00cd
:1086200000c8a8000100370000c8a900f50f20000d
:10863000850f520003003200b4458000e10f520064
:1086400002003a0000e8a8000000060000e8a900c7
:1086500000000600889fbe00c49f200014427800de
:108660008442e900e1cf520004003600e44f52009a
:1086700002003200e54f520014003a00e38120006e
:108680006a814100c1408000b0408000740d070045
:10869000c38320006a814100c1408000b040800057
:1086a0006f0d0700e38620006a814100c140800011
:1086b000b04080006a0d0700038a20006a814100f3
:1086c000c1408000b0408000650d0700fc49ed000e
:1086d000e14f5000c0003e00e49f200014427800ab
:1086e000e04f520049003a00aac8bf006140600054
:1086f000e1036000c83bdd00044080000480a1006d
:108700008703720066458000610363004933dd0022
:108710000790a1000683730075458000e182620026
:10872000ca2add0006a0a1008502730084458000ee
:10873000610262004b22dd0005b0a10004827200dc
:1087400095458000e1826200cc2add0004c0a100d2
:108750000502720004408800c222ab000a00320009
:108760000410b20008003200844b8000954b80005a
:10877000e40f5200e08f5a002400360061025200dc
:10878000e0825a000b003700c222ab001600320014
:108790000128ab0014003200844b8000954b800010
:1087a000ef0f5200e08f5a0018003e0061024200b5
:1087b000e0824a00844b8800954b88008400780052
:1087c00060002000b213070020002000de13070025
:1087d00000e0230091042000e613070020002000a1
:1087e000d5130700090037008c0f070000408000f8
:1087f0004900de00614060008f0f070000408000ec
:108800004a00de0061406000980f0700464180008a
:10881000564088005041800060408800348220002b
:1088200014427800ef4f520026003e000482fb0005
:108830008403e90087b2de00e18262000f003200ab
:108840008402780012002000030020000204be0011
:10885000850078008100e90003003300080444002b
:1088600089844c00fbff3700080373008502e80091
:10887000ef8f5200f5ff3400564088008783de00fa
:10888000e18363000f003200654080001600200085
:10889000070020000600be00040178000201e90084
:1088a000030033000000400081804800fbff3700d8
:1088b000808272000402e800ef0f5200f5ff3400de
:1088c00065408800840c200055408000848f520051
:1088d000010034005440880084f32f00554080008c
:1088e000848f520001003d0054408800840c200019
:1088f00065408000848f520001003400644088008d
:1089000084f32f0065408000848f520001003d00f9
:1089100064408800824b80006140800050408000ad
:10892000c90f07003442800045418000850f520086
:1089300007003a005541800046428000850f5300f1
:1089400003003a004a08f8000408f9000100370063
:10895000244088001484200014427800ef4f520015
:1089600014003e00254080000482fb000403e9005f
:1089700006abde00610363000e003200160020002b
:10898000070020000600be00040178000201e90093
:10899000030033000000400081804800fbff3700e7
:1089a000808272000402e800ef0f5200f5ff3400ed
:1089b0002540880024408000e00f5200020034006f
:1089c000140020002440880024408000e00f520062
:1089d00001003d0004a8ef00c49f2000144278006d
:1089e00064425200e14f52005e003e00244b800082
:1089f000354b8000e00f5200e08f5a0003003a0030
:108a0000004580009ffd070005003700e10f520080
:108a1000e08f5a0002003a000045800015fe070072
:108a2000c222ab002f003200264b8000374b800063
:108a300061024300e0824b00244b8800354b8800e4
:108a4000e10f5200e08f5a00020036006429ef0067
:108a50006629ef00200020003b13070000002500de
:108a6000310c2000431307000004eb000b0037001b
:108a7000200020003013070000402d0001032000db
:108a80003c130700200020002f13070000402d009a
:108a900001032000371307000804e800244b80007e
:108aa000354b80006140b90061034200e0834a0019
:108ab000860f5000878f5800edff39008400780042
:108ac0000000eb00f212070000002500310c20002e
:108ad00028130700200020001713070002a8a90090
:108ae00002c8a900f49f200014427800e04f520011
:108af0000c003a00004080004800de006140600049
:108b0000c60e0700004080004900de0061406000a2
:108b1000c90e0700004080004a00de00614060008e
:108b2000d20e0700004080004500de00614060007a
:108b3000f00e0700004080004400de00614060004d
:108b4000e50e0700004080004700de006140600045
:108b5000f60e0700004080004600de006140600025
:108b6000eb0e07004f04be00000006000002eb0001
:108b7000944088000440780014e8b700b4408800ae
:108b80001ce8b700000006000200fa001cc8bf0085
:108b900003003a00380a07001ce8b7000c00370051
:108ba0000b0a070024c5b300844f500008003a00a8
:108bb0001228ef001c68ef001468ef00b04080003e
:108bc000e00f500002003200bfe807001628ef0057
:108bd0009440800005002000e40f5200e08f5a000e
:108be0006d003e0004600100040037000a003700f9
:108bf00045003700470037005300370020002000b1
:108c0000d1120700fc69ef00c05d2a003f11070088
:108c1000140020005b0037001cc8bf005e0032005b
:108c2000eb090700c4c5b300844f50005a003a0056
:108c30000000eb00a3120700305f2a003311070089
:108c40002400200094408800a2002000030020009f
:108c500060032400e0110700d4538000844a900090
:108c60008582fb00144b90004833dd000503730040
:108c700007002000a64f8800b74f8800a44a900044
:108c80008582fb00344a90004822dd000502720014
:108c900005002000c44f8800d54f880020602a00be
:108ca0001a110700a04f8000b14f8000480add0074
:108cb0004800de0000007200c808de004111070015
:108cc000a04f80003f11070070602a000f110700bd
:108cd000a0602a000d110700c04f8000d14f800016
:108ce000480add004800de0000007200c808de000f
:108cf00034110700c04f800032110700f0602a00d5
:108d00000211070024003700200020008a1207000b
:108d100021003700b4408000e381200093417800b7
:108d20006282200012417800018220009140780088
:108d30001cc8bf00e609070044002000e04f5000b7
:108d400010003200140037000f01e9008f80e900a5
:108d50001cc8bf00180a0700e04f50000e00320088
:108d60006ffa9700e04f520005003a00fffa9700b3
:108d70008582fb00f4408000848f520003003200a3
:108d800024002000944088000300370024002000c5
:108d9000944088002ffe07000080fa0000000600c3
:108da000af02b000889fbe008a9fbe008c9fbe00ad
:108db0008e1f780049812000994478000040eb0024
:108dc00080cf5400ec013a002449800064409000b8
:108dd000a2c0b3000440bc00020078003009b40017
:108de00040409000fce9b70020612a00c71007004e
:108df000fcc9bf000080fb00f2100700f0602a00f1
:108e0000c2100700fcc8bf0080ef9f0010622a005c
:108e1000be1007000fe997000280fb00e910070071
:108e2000f0602a00b91007000945780089457800ec
:108e3000094678008946780099ef9f000847780036
:108e4000a9ef9f009b0137000d84fb00e502200085
:108e500005c4b900080078002a09b40000047800ad
:108e6000c49f2000144278008442e900e1cf520000
:108e7000af003e00e24f520002003a0020632a0099
:108e8000a2100700c49f200014427800e14f520056
:108e900002003a0010642a009c10070020652a0096
:108ea0009a10070018009000c6100700f0602a0012
:108eb0009610070098047800e08f54007c013a0077
:108ec00028129000b8129000e60f5200e08f5a006e
:108ed00071003a0018029000e10f520074013a004c
:108ee000e04f560039003a00e0cf550037003a0015
:108ef000086f900005032000140320001d003700b8
:108f00000e407800a2c0b3000440bc00020078000c
:108f10003009b400e0b79f0010672a0084bf9f00ab
:108f2000f5b79f00791007006fb1970022009000fd
:108f3000a4100700f0602a0074100700efb3970038
:108f400027039000ffb297000fba9700850f5300d8
:108f500003003200840f530004003a00020037007f
:108f60001cc0b300010037001bc0b3008944e800f7
:108f70000e47e800186b900086cf5400e0ff3900e0
:108f8000485f90000e80fb004300dd002c09b40018
:108f900010029000670242004322de00f440880085
:108fa000685a90000482fb00044188002860900009
:108fb00022e8b7007858900023e8b70008609000d6
:108fc00024e8b700850b070026e8b700e04f5500fe
:108fd00037013a00086f90008a447800840320002b
:108fe000160037000e407800a2c0b3000440bc0059
:108ff000020078003009b400e0b79f0010672a0033
:1090000084bf9f00411007006fb1970022009000bd
:109010006c100700f0602a003c1007006fb3970047
:10902000a60290000fba9700848f520001003a0008
:109030001ac0b3008944e8000e47e800986a90001f
:1090400085cf5400e7ff3900485f90000e80fb0099
:109050004300dd002c09b4001002900067024200ba
:109060004322de00e4418800685a90000482fb003d
:10907000f44188002860900040e8b70078589000dc
:1090800041e8b7000860900042e8b700530b0700c2
:1090900044e8b70006013700e20f5200e08f5a00a3
:1090a00003013a0018029000e90f520000013a0053
:1090b00008689000a2c0b3000440bc000200780021
:1090c0003009b4008004780010672a000f100700f0
:1090d000290090003b100700f0602a000b100700e9
:1090e000485f90000e80fb004300dd002c09b400b7
:1090f00010029000670242004322de00044588000f
:10910000685a90000482fb00144588002860900093
:10911000a4e8b70078589000a5e8b7000860900070
:10912000a6e8b7002d0b0700a8e8b700e00037005d
:10913000e4425200e1cf5200dd003e00e44f520015
:1091400002003a00a0682a00f00f0700c49f200028
:1091500014427800e54f520002003a00c0692a002c
:10916000ea0f070098047800e08f5400d0003a001e
:1091700028129000b8129000e20f5200e08f5a00bf
:10918000cb003a0018029000e10f5200a9003a000b
:10919000e04f560042003a00e0cf550040003a0050
:1091a0001fe99700e04f51003d003a00086f900022
:1091b0000503200014032000230037000e40780030
:1091c000a2c0b3000440bc00020078003009b40023
:1091d000e0b79f0010672a0084bf9f00f5b79f008b
:1091e000ca0f07006fb1970022009000f50f07002b
:1091f000f0602a00c50f0700efb397002703900027
:10920000ffb297000fba9700850f53000600320097
:10921000840f53000600320027032000870f5300fd
:1092200005003200060037001cc0b3000400370000
:109230001bc0b3000200370010c0b30090ef9f00c6
:109240008944e8000e47e800186b900086cf540070
:10925000daff3900485f90000e80fb004300dd001c
:109260002c09b40010029000670242004322de0085
:10927000f4408800685a90000482fb000441880092
:109280002860900022e8b7007858900023e8b700e3
:109290000860900024e8b700d00a070026e8b7006d
:1092a000e04f550030003a00086f90008a44780083
:1092b00084032000160037000e407800a2c0b300df
:1092c0000440bc00020078003009b400e0b79f0001
:1092d00010672a0084bf9f008c0f07006fb19700b2
:1092e00022009000b70f0700f0602a00870f0700e8
:1092f0006fb39700a60290000fba9700848f5200b8
:1093000001003a001ac0b3008944e8000e47e800a3
:10931000986a900085cf5400e7ff3900485f9000bd
:109320000e80fb004300dd002c09b4001002900009
:10933000670242004322de00e4418800685a900040
:109340000482fb00f44188002860900040e8b700e8
:109350007858900041e8b7000860900042e8b700f4
:109360009e0a070044e8b7002fe99700e04f51003c
:109370004f003a00086f90008244780016003700d2
:109380000e407800a2c0b3000440bc000200780088
:109390003009b400e0b79f0010672a005b0f070098
:1093a0006fb1970022009000860f0700f0602a003e
:1093b000560f0700efb29700250290009603200099
:1093c000860f520002003a0017c0b300a7ef9f00bb
:1093d0008944e8000e47e800186a900084cf5400e2
:1093e000e7ff3900485f90000e80fb004300dd007e
:1093f0002c09b40010029000670242004322de00f4
:1094000074438800685a90000482fb0084438800fb
:109410002860900072e8b7007858900073e8b700b1
:109420000860900074e8b7006c0a070076e8b7009f
:109430001f003700e90f52001d003a00485f9000fe
:109440000e80fb004300dd002c09b40010029000e8
:10945000670242004322de0004458800685a9000fb
:109460000482fb001445880028609000a4e8b7003f
:1094700078589000a5e8b70008609000a6e8b7000b
:10948000560a0700a8e8b700a008f800e26a2a0018
:10949000821f780060fc2f000f004000dae6070012
:1094a00060fc2f000f004000180f0700e4875700f2
:1094b0008d46e8000fea970084cf560062fe39001f
:1094c0000e4478001fef9700afec9700a06c2a00c5
:1094d0000e0f0700fdc8bf000080fb00390f07001a
:1094e000f0602a00090f0700d48f20001442780092
:1094f000e04f52001f0032000880fb004300dd00f7
:109500002c09b40010009000670040004300de000a
:10951000c0408800dee50700b0408800d208f800af
:109520001a08f900e04f56000200320010c0b300e4
:1095300014e8b700e0cf55000200320010c0b300bd
:1095400014e8b700e04f57000200320010c0b3002b
:1095500014e8b700e04f55000200320010c0b3001d
:1095600014e8b700e0cf54000200320010c0b3008e
:1095700014e8b70014c8bf004f0778004f06be00bc
:109580004f05be004f04be00af02b1000000060050
:1095900000a0fe003600f800849fbe00869fbe003b
:1095a000889fbe00692480008c24ef00181680007c
:1095b00062046400b8003a00244b8000354b800000
:1095c000e10f5200e08f5a00b3003a00c49f200020
:1095d0001442780064425200e14f5200ae003e0057
:1095e00010c0b300ffe9b700c902a800c8e2a90093
:1095f000c9c2a900c9e2a900c8a2a800044080000d
:109600004922de000482ea0061026200e102620097
:10961000c72bdd00661680000670a10007037300eb
:10962000661688004e2bdd006516800005e0a1005f
:109630008682720065168800cf22dd0064168000e5
:1096400004f0a1000502720064168800fc0c0700fb
:10965000044080004822de000482ea0061026200c9
:10966000e1026200c72bdd00661680000670a100d3
:1096700007037300661688004e2bdd006516800018
:1096800005e0a1008682720065168800cf22dd0009
:109690006416800004f0a1000502720064168800c0
:1096a000e70c0700044080004a22de000482ea0042
:1096b00061026200e1026200c72bdd0066168000d5
:1096c0000670a10007037300661688004e2bdd00ac
:1096d0006516800005e0a10086827200651688008c
:1096e000cf22dd006416800004f0a10005027200a4
:1096f00064168800d20c0700044080004b22de0074
:109700000482ea0061026200e1026200c72bdd0010
:10971000661680000670a1000703730066168800b5
:109720004e2bdd006516800005e0a10086827200e8
:1097300065168800cf22dd006416800004f0a100c9
:109740000502720064168800bd0c0700044080000a
:109750004d22de000482ea0061026200e102620042
:10976000c72bdd00661680000670a100070373009a
:10977000661688004e2bdd006516800005e0a1000e
:109780008682720065168800cf22dd006416800094
:1097900004f0a1000502720064168800a80c0700fe
:1097a000044080004c22de000482ea006102620074
:1097b000e1026200c72bdd00661680000670a10082
:1097c00007037300661688004e2bdd0065168000c7
:1097d00005e0a1008682720065168800cf22dd00b8
:1097e0006416800004f0a10005027200641688006f
:1097f000930c0700144080004622de000482ea0039
:1098000061026200e1026200c72bdd006616800083
:109810000670a10007037300661688004e2bdd005a
:109820006516800005e0a10086827200651688003a
:10983000cf22dd006416800004f0a1000502720052
:10984000641688007e0c0700cce2a800cdc2a800f8
:10985000cde2a8007a0c0700cce2a900cdc2a90095
:10986000cde2a900760c0700cce2a800cdc2a8008a
:10987000cde2a800720c0700c902a800c8e2a80047
:10988000c9c2a800c9e2a800c8a2a8000840780080
:10989000ffe9b700bb0037001816800062046400bf
:1098a000b8003a00fc49ed00e14f5000b5003e0021
:1098b00010c0b300fee9b700c902a800c8e2a900c1
:1098c000c9c2a900c9e2a900c8a2a800044080003a
:1098d0004922de000482ea0061026200e1026200c5
:1098e000c72bdd00661680000670a1000703730019
:1098f000661688004e2bdd006516800005e0a1008d
:109900008682720065168800cf22dd006416800012
:1099100004f0a1000502720064168800480c0700dc
:10992000044080004822de000482ea0061026200f6
:10993000e1026200c72bdd00661680000670a10000
:1099400007037300661688004e2bdd006516800045
:1099500005e0a1008682720065168800cf22dd0036
:109960006416800004f0a1000502720064168800ed
:10997000330c0700044080004a22de000482ea0023
:1099800061026200e1026200c72bdd006616800002
:109990000670a10007037300661688004e2bdd00d9
:1099a0006516800005e0a1008682720065168800b9
:1099b000cf22dd006416800004f0a10005027200d1
:1099c000641688001e0c0700044080004b22de0055
:1099d0000482ea0061026200e1026200c72bdd003e
:1099e000661680000670a1000703730066168800e3
:1099f0004e2bdd006516800005e0a1008682720016
:109a000065168800cf22dd006416800004f0a100f6
:109a10000502720064168800090c070004408000eb
:109a20004c22de000482ea0061026200e102620070
:109a3000c72bdd00661680000670a10007037300c7
:109a4000661688004e2bdd006516800005e0a1003b
:109a50008682720065168800cf22dd0064168000c1
:109a600004f0a1000502720064168800f40b0700e0
:109a70000488d5000082ea0061026200e10262000f
:109a8000c72bdd00661680000670a1000703730077
:109a9000661688004e2bdd006516800005e0a100eb
:109aa0008682720065168800cf22dd006416800071
:109ab00004f0a1000502720064168800e00b0700a4
:109ac000244080000482ea0061026200e102620038
:109ad000c72bdd00661680000670a1000703730027
:109ae000661688004e2bdd006516800005e0a1009b
:109af0008682720065168800cf22dd006416800021
:109b000004f0a1000502720064168800cc0b070067
:109b1000cce2a800cdc2a800cde2a800c80b070087
:109b2000cce2a900cdc2a900cde2a900c40b070078
:109b3000cce2a800cdc2a800cde2a800c00b07006f
:109b4000c902a800c8e2a800c9c2a800c9e2a800ca
:109b5000c8a2a8002840880008407800fee9b700a5
:109b6000fde9b700004080004800de006140600071
:109b7000aa0a0700004080004900de006140600042
:109b8000ad0a0700692488008660a9004f04be0062
:109b90004f03be004f02be003600f9000080fe00f9
:109ba000004006000042eb0004407800f2e8b700f5
:109bb00016c0b30006407800f3e8b7008002eb005f
:109bc000054788001547880005407800f8e8b70089
:109bd00004407800f9e8b700fae8b700fce8b700fd
:109be00006407800fde8b70055478800044078003b
:109bf00000e9b70002e9b7008547880001e9b7002e
:109c0000d5e8b700d6e8b700d7e8b700d8e8b7007e
:109c1000d9e8b700dae8b7006033b80056488800e2
:109c2000674888003648880047488800964888007a
:109c3000a7488800764888008748880022e9b7004e
:109c400020e9b700f548880021e9b700d648880028
:109c5000e7488800b6488800c7488800254888003b
:109c6000000006008002780020002000e08f5200f3
:109c70008a00320014922000144278000482fb0013
:109c800016002000070020000402e9000300330052
:109c90000603430087834b00fbff3700d000200002
:109ca0005248800063488000860f5100878f59001a
:109cb0007a003d0080002000a48d2000144278002e
:109cc000e04f520075003a00948d20001442780055
:109cd000e04f520071003a0090002000848d200077
:109ce00014427800e04f52006c003a00748d20005e
:109cf00014427800e04f520068003a00a0002000b3
:109d0000648d200014427800e04f520063003a0056
:109d1000548d200014427800e04f52005f003a005a
:109d2000c68f2000164378000680fb00e402200066
:109d30000481b900020078002a09b400000278000a
:109d40000643e80006407800fce8b70015039000e1
:109d5000a50390002612980037129800e2034200f3
:109d6000409020000f000900b01b7800b68f200043
:109d70001643780036629800568f2000164378000c
:109d8000066a9800179020009743780007407800f3
:109d9000f5e8b70006c35300166a9800768f2000d6
:109da00016437800266a9800f78f200097437800c2
:109db00007407800f7e8b70006c35300366a9800fa
:109dc000668f200016437800466a9800478f20006f
:109dd0009743780007407800f6e8b70006c35300c1
:109de000566a9800f04880004300dd002c09b4005a
:109df00027922000974378008783fb00169220006b
:109e0000164378000683fb0006bbb9009502780074
:109e1000c42ade00ef826200e98f52000d0032009a
:109e2000eb8f520003003200e88f520018003a0016
:109e30001000370025002000050a7800e04290005d
:109e40002562980030029000060342003600980018
:109e50000e00370015002000050a7800c04390006e
:109e60002762980020029000060342002600980016
:109e700006003700000aeb00a0429000256298001f
:109e80001002900006034200160098000000050032
:109e900035002000050a78000000eb0000000600f5
:109ea0009042780063c262001a003200100378000a
:109eb000e3026300e38f520001003a0044c0b300a4
:109ec0008482fb008502e800e0c27a00e0cf520005
:109ed00010003d000c0037000483fb004333dd001d
:109ee000062bdd00cfb3de0010019000a001900032
:109ef0000603710087837100160098002700980000
:109f00000442e80001003700f50f2000e44f520042
:109f1000f1ff3a000000060000037800348f2000b3
:109f2000144278008442e80005407800f3e8b70066
:109f30002549800004407800e2c0b3000440bc0022
:109f4000028142003619780026117800568f2000d1
:109f50001643780066419800568f2000164378001b
:109f600017902000174313007641980001c9bf00e5
:109f7000f5e8b700e68f20001643780046499800c0
:109f80000043eb0006407800fee8b7003649980031
:109f90002648800026019800c78f2000974378004c
:109fa00007499800fbc8bf0020499800fbc8bf00c4
:109fb000e2c0b3000440bc0082824200b44a980070
:109fc000258f2000954278000583fb00974980008b
:109fd000fbc8bf0080737b008542e8000540780025
:109fe000f2e8b70004407800fbe8b7000000060084
:109ff000fbc8bf00e2c0b3000440bc000200780010
:10a000002409b400004a9000c58f200015421200b8
:10a0100014489800f248ed00f2e8b7000080fb0019
:10a020009449800064427800fbc8bf00fee8b70096
:10a0300004407800fbe8b700000006000600fa00c4
:10a04000889fbe008a9fbe008c9fbe000004be0099
:10a05000020578008345780021002000e00f5400bd
:10a0600007033200e08f540005033200208d2000ea
:10a07000280009000018eb00cafe07000b4078001a
:10a08000d4e8b7009a468800880278000902780070
:10a090008000eb0015417800e2ef9f00e343610090
:10a0a0007fb397006300630046c0b300e30f500026
:10a0b00001003200074378008683fb008783ea00b3
:10a0c00007024200ffb397004238de0063006000e1
:10a0d000e10f500024003200e20f50003b0032003c
:10a0e000e00f500059003a004439de006f01610072
:10a0f000cf91de0068015100e0815900e40f51006a
:10a10000e08f590051003e0002600100140037004a
:10a110001300370002003700110037000900370034
:10a12000f368ec00f248ec00f2e8b700978f2000eb
:10a1300097437800874f500044003600f9e8b70095
:10a1400042003700278f2000974378000740e9003e
:10a15000f2e8b700e0cf5300390032003b0037008f
:10a16000fc68ec0039003700c43bde00ef8363007d
:10a17000ea8f530006003200eb8f53000c003200d0
:10a18000e88f530031003a00fd68ec002f003700e3
:10a19000f848ec00f8e8b700a78f20009743780054
:10a1a000874f500029003600fae8b7002700370033
:10a1b000f848ed00f8e8b700a78f20009743780033
:10a1c000874f500020003e00200037004439de0059
:10a1d0006f016100cf91de00e90f5100e08f59005f
:10a1e0001a003e0002600100090037000a00370033
:10a1f000090037000e0037000f0037000e0037004f
:10a20000120037000600370007003700060037004d
:10a210000269ec000d003700f028ec000b0037005d
:10a220000069ec0009003700ea28ec00070037005d
:10a23000e228ec0005003700e028ec0003003700be
:10a24000310020000100370041002000e00f5200e3
:10a25000040032000683fb000603e8008682420009
:10a260008cff370001057800e08f500084023a002f
:10a2700051002000248f200014427800e04f52004b
:10a280007f023a00338f2000934178006100200064
:10a29000e1cf51007a023200c78f20009743780047
:10a2a00071002000e0cf5300750232008647800025
:10a2b000610263008100200071023a00544780006f
:10a2c000e1026200910020006d023a000547800023
:10a2d00061816200a100200069023a000603d100fa
:10a2e00020902000104343000640780002e9b700a8
:10a2f0000402d10001902000114242000440780085
:10a3000000e9b7008502d100114780008182420038
:10a31000154788008783fb00e102200001beb900d9
:10a3200003407800e2c0b3000440bc008c0341004d
:10a33000d18f2000914078008180fb00c308dd00b0
:10a340008183430006407800a2c0b3000440bc00f3
:10a3500082834300a68f2000164378000683fb000b
:10a360004233dd00850243000482fb000482420088
:10a370004222dd00968f2000164378000683fb0002
:10a38000060242000402420084854300a049800086
:10a39000e00f500001003200cbe207000b00780014
:10a3a0003be20700a049880040112a00570b070034
:10a3b0000b007800830b070080132a00530b070063
:10a3c000a449800011002000e00f52002c0232004e
:10a3d00024498800f3c8bf00e2c0b3000440bc00b9
:10a3e0000202420054498800c28f200012417800c6
:10a3f0000281fb00e50220000591b9000201420044
:10a4000062498800d48f2000144278000482fb0047
:10a410004322dd00040241008449880002c9bf00d4
:10a42000a2c0b3000440bc0002024200744988008c
:10a4300005902000954278008582fb00c32add004c
:10a44000050242003449880015478000c32add0018
:10a450000502420094498800958f200095427800bb
:10a460008582fb0085824200050242004449880043
:10a47000ccfd070024498000000aeb00341278006c
:10a480008042eb00354a9800054a980065429800e2
:10a49000454a9800254a9800154a98007542980048
:10a4a0008002eb0025029800644980003502980084
:10a4b0001502980025029800050a7800b0132a00ba
:10a4c000120b070098407800e1ef9f0063c2600024
:10a4d0007fb19700e30361004bc0b300e38f5300eb
:10a4e00001003200844578000804e8000801780083
:10a4f0006022b8000043eb000d00370032407800c6
:10a500000080fb00010020008681fb00c319dd00f4
:10a510008301e9000300330000004000818048000f
:10a52000fbff370000027200818272000643e800e0
:10a530008b4f5300f1ff39000b83fb0006044400ee
:10a5400084bf9f0095bf9f007fb397004230de001d
:10a5500063006000e10f50001b003200e20f50006a
:10a560008f003200e00f5000a9013a004433de00b2
:10a570006f036300cfb3de0068035300e0835b002a
:10a58000e40f5300e08f5b00a1013e000660010074
:10a5900004003700030037000600370001003700d1
:10a5a0000700370072805700aefd0700800078007a
:10a5b000950137007080570057fe0700940137005f
:10a5c0008bfe0700920137004433de006f03630007
:10a5d000cfb3de00eb0f5300e08f5b008c013e0039
:10a5e000066001000b0037000c0037001200370036
:10a5f000180037001e0037002400370084013700a0
:10a6000025003700290037004b0037004d00370088
:10a6100059003700244888007d01370072805700b8
:10a620001ffe07000fba97009fba970034488800b2
:10a6300045488800760137007280570018fe0700f1
:10a640000fb897009fb8970050488800614888006d
:10a650006f0137007280570011fe07000fba970094
:10a660009fba9700744888008548880068013700c1
:10a67000728057000afe07000fb897009fb8970036
:10a6800090488800a148880061013700b4488800dc
:10a69000c54888005e0137000440780021e9b70012
:10a6a000e04f52007c01320059013700e00f5200a8
:10a6b000e08f5a007a013200d78f2000974378004c
:10a6c000604980000043eb00010037000643e800ca
:10a6d000874f5300070031008680fb00c308dd0070
:10a6e0006081780003002000840f5100858f59009d
:10a6f000f6ff3a00874f53000a003a008683fb00ba
:10a70000c33bdd00870340000640e800fde8b700da
:10a71000840b78008400200094039800a403980020
:10a72000b40398000ff0970020e9b7000683fb0000
:10a73000f6488800360137000440780022e9b70067
:10a7400033013700848f2000144278000480fb001e
:10a750004500dd002809b400419020000f000900e9
:10a76000311878000002b1000442e800044078008b
:10a77000f8e8b70026013700f848ed00f8e8b70020
:10a780000080fb004500dd0044498000419020002e
:10a79000000142000f000900b21878001c013700c8
:10a7a0004430de006f006000cf80de00e90f500013
:10a7b000e08f580016013e000060010009003700dc
:10a7c000230037005a003700940037009d003700ff
:10a7d000b40037000e013700cc003700d800370036
:10a7e000ef003700149020001442780004407800f5
:10a7f000a2c0b3000440bc00020078003009b400dd
:10a80000000378000442e8000440780001e9b70042
:10a81000004beb00ffb0970063826000e30f520033
:10a8200006003a001fb99700120398000fba97006c
:10a83000f40fb20024039800f5003700244880008c
:10a84000140398008fba970025039800f000370092
:10a85000968d200016437800e04f53002700320009
:10a86000149020001442780004407800a2c0b30085
:10a870000440bc00020078003009b40000037800f6
:10a880000442e8000440780001e9b70014c0b300b6
:10a89000044b7800ffb0970063826000e30f520022
:10a8a00006003a001fb99700120398000fba9700ec
:10a8b000f40fb200340398000400370024488000ed
:10a8c000140398008fba9700350398009602900001
:10a8d0002101200024478000848f520001003a00ab
:10a8e0008a0078006447800044039800b602900014
:10a8f000850f52003900310037003700e38f5300d5
:10a9000004003a0025478800f40fb200744788001d
:10a91000040037000409f800e408f9000fbb9700b1
:10a920007647880010c0b300dae8b700b8003700f7
:10a93000a68d200016437800e04f53002a00320015
:10a94000149020001442780004407800a2c0b300a4
:10a950000440bc00020078003009b4000003780015
:10a960000442e8000440780001e9b70014c0b300d5
:10a97000044b7800ffb0970063826000e30f520041
:10a9800006003a001fb99700120398000fba97000b
:10a99000f40fb200440398000400370024488000fc
:10a9a000140398008fba9700450398009602900010
:10a9b0002101200024478000848f520001003a00ca
:10a9c0008a0078007447800034039800c602900023
:10a9d000848f52000100310031012000d968ef005e
:10a9e000da68ef0088003700e38f530004003a0074
:10a9f00025478800f40fb200644788000400370040
:10aa00000409f800e408f9000fbb970066478800c6
:10aa100010c0b300d9e8b7007d003700448f200094
:10aa2000144278000480fb004300dd002609b400d6
:10aa3000800278000442e80004407800f4e8b7009f
:10aa40003b003700568d200016437800e04f53003e
:10aa500010003200448f2000144278000480fb0074
:10aa60004300dd002609b400800278000442e800bb
:10aa700004407800f4e8b70014c0b300844a7800ba
:10aa80008fb89700a1029800e2468000b2029800b9
:10aa900017003700f446880010c0b300d6e8b700ae
:10aaa0005b003700668d200016437800e04f5300ae
:10aab00012003200448f2000144278000480fb0012
:10aac0004300dd002609b400800278000442e8005b
:10aad00004407800f4e8b70014c0b300844a78005a
:10aae0008fb89700b1029800f2468000a202980049
:10aaf000d668ef00d568ef0045003700e4468800cf
:10ab000010c0b300d5e8b70041003700f48f200033
:10ab1000144278000480fb004300dd002e09b400dd
:10ab2000800278000442e80004407800ffe8b700a3
:10ab3000804aeb008fb897009102980034003700ec
:10ab4000768d200016437800e04f5300100032004d
:10ab5000f48f2000144278000480fb004300dd00e5
:10ab60002e09b400800278000442e8000440780016
:10ab7000ffe8b70014c0b300844a78008fb897008c
:10ab8000a102980032478000b202980017003700f7
:10ab90004447880010c0b300d8e8b7001c00370055
:10aba000868d200016437800e04f530012003200db
:10abb000f48f2000144278000480fb004300dd0085
:10abc0002e09b400800278000442e80004407800b6
:10abd000ffe8b70014c0b300844a78008fb897002c
:10abe000b102980042478000a2029800d868ef00a6
:10abf000d768ef00060037003447880010c0b30064
:10ac0000d7e8b70002003700e08f50001c003a0080
:10ac10008b85fb008b85ea008b84440029fe3a007b
:10ac20006649800015c0b300100037000582fb00a4
:10ac30004322dd000402430094039000e88f530098
:10ac400001003a0019029800a4039000e88f530015
:10ac500001003a0029029800b4039000e88f5300e5
:10ac600001003a00390298008542e800d48f2000a4
:10ac70001442780084cf5200ecff39008a0078003b
:10ac8000010078004f06be004f05be004f04be0015
:10ac90000080fa0000000600f1002000f8ff3700f5
:10aca00001012000f6ff3700889fbe008a9fbe008a
:10acb0008c9fbe008002780002037800e08f510074
:10acc0005b0032000504780008f0a7000804ea00e1
:10acd0000804e9004f44de0055003a00056d90007d
:10ace0008003eb0019c0b3004e0037000a40780023
:10acf000a2c0b3000440bc00020078003009b400d8
:10ad00008006780012002000e08f5000060032001c
:10ad10001d0190000281680002f0a7000201ea0014
:10ad20000201e9004f11de008045eb009dcf1500c8
:10ad300024003200bd0590008b0f5300190039002c
:10ad40004d0690008c0f530016003e008b055300fb
:10ad500087894500e00f5200100032000886fb0092
:10ad60000c06e800956d90008b85fb008b0f56005c
:10ad700009003a00cd0590008b0f530006003a0001
:10ad80008565900087c55500e1cf5500020036006b
:10ad90000b4a780001003700094a7800e04f510063
:10ada00025003a00cd0590008b05e8003d0190009c
:10adb0000280550000f0a7000000ea0080834300f5
:10adc000160037002d009000800f530012003a004b
:10add00087097800e00f52000d0032008885fb00e3
:10ade0008b05e800156890000080fb00808f5500ff
:10adf00006003a000560900007405000e14f500007
:10ae000002003600004a780001003700094a780045
:10ae1000e04f510008003a008703e8000a45e800c7
:10ae20000844e80015689000804f5400afff3900d7
:10ae30000040eb000100370010c0b3004f06be0019
:10ae40004f05be004f04be0000000600889fbe00f4
:10ae50008a1f780050152a00ac080700201a2a0023
:10ae6000aa080700f3c8bf000080fb00d508070050
:10ae7000301b2a00a5080700f9c8bf000080fb00ae
:10ae8000d0080700401c2a00a0080700fdc8bf002a
:10ae90000080fb00cb080700101d2a009b0807005c
:10aea000fcc8bf000080fb00c6080700201e2a0067
:10aeb0009608070001c9bf000080fb00c108070019
:10aec0008044eb0037003700301f2a008f0807004e
:10aed000f0202a008d0807000984fb000800780094
:10aee000b80807006e42b900040078002409b400d5
:10aef0000004780040222a00840807001800780027
:10af0000b0080700d0232a0080080700280090001e
:10af1000ac08070060252a007c0807006840900004
:10af20000080fb00a7080700f0262a00770807002a
:10af3000784090000080fb00a208070080282a00cb
:10af400072080700084890000080fb009d08070079
:10af5000102a2a006d080700184890000080fb00a6
:10af600098080700a02b2a006808070028489000ce
:10af70000080fb0093080700302d2a0063080700bb
:10af8000384890000080fb008e080700c02e2a0081
:10af90005e080700484890000080fb008908070011
:10afa0008944e800348f20001442780084cf540094
:10afb000c5ff39008044eb002400370050302a00e0
:10afc0005208070000322a00500807000984fb00dd
:10afd000080078007b0807004340dd002c09b4001e
:10afe00000047800e0322a004808070018007800c2
:10aff0007408070018029000e00f520002003200af
:10b00000c0332a0041080700180090006d080700af
:10b0100028029000e00f520002003200a0342a0003
:10b020003a080700280090006608070038029000e0
:10b03000e00f52000200320080352a00330807007a
:10b04000380090005f0807008944e800d48f200092
:10b050001442780084cf5400d8ff39008044eb00bc
:10b06000ea0220004200370050302a00270807007b
:10b0700060362a00250807000984fb0008007800d4
:10b08000500807000ac2b900040078002a09b40079
:10b090000004780070372a001c08070018007800a8
:10b0a0004808070080382a00180807002860900028
:10b0b0000080fb004308070090392a0013080700ae
:10b0c000785890000080fb003e080700a03a2a0054
:10b0d0000e080700386090000080fb003908070068
:10b0e000b03b2a0009080700281090003508070027
:10b0f000c03c2a0005080700086890000080fb009b
:10b1000030080700d03d2a000008070018689000aa
:10b110000080fb002b080700e03e2a00fb07070029
:10b1200010402a00f90707001800900025080700c2
:10b1300020412a00f5070700785890000080fb00a6
:10b140002008070040422a00f007070068589000d6
:10b150000080fb001b08070040432a00eb070700a4
:10b16000086090000080fb00160807008944e80092
:10b17000c48f20001442780084cf5400baff3900f5
:10b1800050302a00e107070070442a00df0707005b
:10b190000980fb000b0807000044eb00210037008a
:10b1a00008407800a2c0b3000440bc0082047800cc
:10b1b0008449800064c27c00e04f520011003200dc
:10b1c00070452a00d1070700e0472a00cf07070093
:10b1d000090078003009b4000002780044009000b3
:10b1e000f807070010482a00c80707000900780080
:10b1f0003009b4000002780034009000f107070025
:10b200000200370030482a00c00707000900780014
:10b210003009b4008004780029009000e907070095
:10b220000844e8001490200014427800844f540031
:10b23000dbff39004f0578004f04be000000060018
:10b24000881f7800a493200014427800804f520099
:10b250000f003a000a0037001bdf07004029ef000b
:10b26000030037001004780017df0700e853880058
:10b27000e0538000e00f5000faff3a00040037006e
:10b28000004a8000e00f5000f3ff3a00f8ff37005b
:10b290004f04780000000600889fbe008a9fbe0011
:10b2a0000085fb00c802200008d4b9006e024400eb
:10b2b0006993200069027a000402d10061426200b1
:10b2c0002a0032007482440008024200004aeb0067
:10b2d000040220000902420008024200004aeb007a
:10b2e000a40220000802420069427a00640544007a
:10b2f0008a82440095429000851f78008043eb00cd
:10b300000003eb00860278000482fb0086017800cf
:10b3100000c1eb0011c2b30069407d0040ef07009f
:10b320008f87e90070824400e04f50000b0032002c
:10b330000804420074c5b300044c780044c0b30054
:10b34000144498006022b8000001eb002126200080
:10b3500069407d00860607001a0037000804420095
:10b3600074c0b30014449800160037007002440003
:10b3700069427a0064044400e04f520004003a003d
:10b380006022b8000001eb00e12520000300370037
:10b390006022b8000001eb002126200069407c00fb
:10b3a00073060700c402200004d5b900649420008d
:10b3b0000a0242007205450065932000e5427d00c7
:10b3c000154298004f05be004f04be000000060065
:10b3d00080427800a49320001442780020c5b30076
:10b3e000854f52001d003a001d0037007494200064
:10b3f000144278000482fb00050020006102520024
:10b40000e0825a00e80f5200e08f5a0010003e0020
:10b4100004600100080037000d0037000600370007
:10b420000d0037000a00370009003700060037001a
:10b430000500370002003700a0c5b3000000060079
:10b44000d0c5b30000000600e0c5b3000000060050
:10b4500090c5b30000000600c0c5b30000000600a0
:10b460000440780092e6070004c3b300844f500004
:10b47000faff3a00ddff3700881f7800244a800079
:10b480004522de00614262000044eb00e14f5200c1
:10b490000600320008003700a89320001844780006
:10b4a000e04f54000100320044a9a8000840780091
:10b4b0004f047800000006003ac9bf00c4ff07002f
:10b4c000c4c5b300844f5000f8ff3a00f2ff3700c4
:10b4d000881f780080427800814378000404780057
:10b4e000a69320001643780021c5b300854f530072
:10b4f0002b003a002d00370014027800e00f5200b4
:10b5000003003200844a900082cf5200faff3a00d2
:10b51000f453880031c5b30075942000954278003b
:10b52000e4cf52001e003a00a59420009542780016
:10b53000e0cf52001a003a005029ef00784a880004
:10b54000e44090000140780052e9b70003407800e1
:10b5500053e9b7008783fb00674a88000240780000
:10b5600054e9b7000540780046e9b7000382fb00c4
:10b5700005002000080178000640780015e9070062
:10b5800080407800e0cf500003003a0010c0b300c4
:10b590004ae9b700020037000140780046e9b700e9
:10b5a000014078004f04780000000600e45380005a
:10b5b000f4538800d1ff3700a49320001442780090
:10b5c000804f52001000320024c5b3008448780038
:10b5d0000049eb0010c0b300000006006494200096
:10b5e00014427800844878000495200014427800c2
:10b5f000044978004ac9bf000080fb000000e90050
:10b600004f00de0000000600749420001442780011
:10b61000e04f5200f1ff3a00ebff3700a493200007
:10b620001442780025c5b300804f52000d003a0047
:10b630000e00370095027800e08f520003003200c0
:10b64000054b9000814f5300faff3a00f5538800f4
:10b65000e54090000440780097e707004a69ef0052
:10b660008042eb000540780000000600e5538000b2
:10b67000f5538800f0ff37000042780020c5b30082
:10b68000a59320009542780084cf520009003a002b
:10b6900009003700e0c0b3004469b7004429a8009e
:10b6a00040c0b30048e9b7000040eb00fafe0700d5
:10b6b0000040eb0000000600749420001442780063
:10b6c000e14f5200f3ff3e0080c5b30000000600ca
:10b6d00000000600889fbe00804378008342780007
:10b6e00004037800a99320009944780023c5b3008f
:10b6f00087cf54003b003a003d0037001402780029
:10b70000e00f520003003200844b900082cf5300c0
:10b71000faff3a00f453880033c5b3007794200051
:10b7200097437800e4cf53002e003a00689520003c
:10b7300018447800e04f54002a003a005c29ef00da
:10b74000d64a8800f4439000074078005ee9b700cd
:10b75000054078005fe9b7008181fb000390a000fd
:10b76000c34a88000240780060e9b70008407800ca
:10b7700046e9b700e0cf53000c003a00b493200034
:10b7800014427800841f78008582fb000282fb004f
:10b7900092c0b30011c2b3000940780020ee070048
:10b7a000804178008f87e900070037000582fb00a1
:10b7b00005002000060178008740780009407800e5
:10b7c000e2e8070080417800e0cf510003003a0032
:10b7d00010c0b30056e9b7000200370003407800fc
:10b7e00046e9b700034078004f04be0000000600a1
:10b7f000e4538000f4538800c1ff3700a493200075
:10b8000014427800804f52001000320024c5b3006b
:10b81000844878000049eb0010c0b3000000060027
:10b82000649420001442780084487800c495200075
:10b83000144278000449780056c9bf000080fb001c
:10b840000000e9004f00de000000060074942000b4
:10b8500014427800e04f5200f1ff3a00ebff37004e
:10b860000200fa00889fbe0000447800084078007b
:10b8700081ff0700b0ff9f00e04f500010003a002a
:10b88000e9c5b3007eea070008407800d0fe070053
:10b89000b0ff9f00894f5000faff320066815700c9
:10b8a000e580570008407800d4ff07000042780088
:10b8b00070c5b300e04f5200010032003ff897001e
:10b8c0004f04be000080fa0000000600a493200090
:10b8d0001442780025c5b300804f52000d003a0095
:10b8e0000e00370095027800e08f5200030032000e
:10b8f000054b9000814f5300faff3a00f553880042
:10b90000f540900004407800ebe607005669ef0030
:10b910008042eb000540780000000600e5538000ff
:10b92000f5538800f0ff3700ea874700889fbe0084
:10b930008a9fbe008c9fbe008e1f78000003780097
:10b940000107780082047800030678000404780078
:10b95000880578000bf0a7008b05ea008b05e9004d
:10b96000cf5dde000c02780004f0a7000402ea00bc
:10b970000402e9004f22de0004c275000482fb00cd
:10b98000850578000bf0a7008b05ea008b05e90020
:10b99000cf5dde008b0572000040eb00ed02200061
:10b9a00032003200370037000dd9b90002007800ac
:10b9b0002a09b40000057800908f14002a003a008c
:10b9c00074825700f68157000e01780086007800d7
:10b9d00085bf9f00f6b79f00b3fc07008fba9700a2
:10b9e0007fb39700e04f50001f0032006a0a9000ba
:10b9f0004322dd00040078002c09b4000003780025
:10ba0000164e78002a639000afeb9700874a4300f8
:10ba100065498000e08f540003003a000482420030
:10ba2000140290000b003700e18f540007003a0029
:10ba30000482420024029000670242004322de009a
:10ba4000044c7800094078000e0037000482420060
:10ba500034029000670242004322de00044c78006a
:10ba600010c0b300070037008b05e800c48f20002a
:10ba7000144278000482fb00848f5500caff39000d
:10ba80000040eb004f0778004f06be004f05be0098
:10ba90004f04be00af00b10000000600ee87470073
:10baa000889fbe008a9fbe008c9fbe008e1f7800bc
:10bab000d0b79f0081037800020478000306780065
:10bac00084047800890578000bf0a7008b05ea0054
:10bad0008b05e900cf5dde000c02780004f0a700c2
:10bae0000402ea000402e9004f22de0004c27500ed
:10baf0000482fb00860578000bf0a7008b05ea00a6
:10bb00008b05e900cf5dde008b0572000502780031
:10bb100004f0a7000402ea000402e9004f22de005c
:10bb2000848575000040eb00ed0220002e0020000f
:10bb300040003200440037000b80fb000d81b9004b
:10bb4000020078002a09b40000057800900f140064
:10bb500037003a00201290000e02620034003200da
:10bb6000705a9000e14f5200310032007a82570043
:10bb7000f881570007017800dfb09700f5b79f0004
:10bb800086bf9f00e7b79f0047fc0700ffb2970002
:10bb90000fbb9700efb39700e04f50002400320036
:10bba0006a0a90004322dd00040078002c09b400ea
:10bbb00080037800174e7800fa5b9000074b7800fe
:10bbc0007a5b90000683fb008feb970007b3b90008
:10bbd0002a609000864a400065498000e00f5400ca
:10bbe00003003a0004824200140290000b00370068
:10bbf000e10f540007003a00048242002402900042
:10bc0000670242004322de00844c7800084078003e
:10bc10000d003700048242003402900067024200a7
:10bc20004322de00844c780010c0b30006003700c9
:10bc30008b45e800c48f20001442780084cf550063
:10bc4000bdff39000040eb004f0778004f06be00f3
:10bc50004f05be004f04be00ef00b100000006001b
:10bc6000889fbe008a9fbe008c1f78000006780067
:10bc700081047800e00f56005200320093029000d9
:10bc8000e08f5200050032001c4078000083fb006a
:10bc90000042eb00868f52004b003a000042eb005e
:10bca000938f140048003a00c34290008582fb0045
:10bcb0000504e900e34390008783fb0053439000b1
:10bcc0000683fb0006bbb900860344008600200003
:10bcd000110009008603d800000378008000eb0003
:10bce00018002000890f530030003600360037005e
:10bcf000432dde00e7846200d34390000783fb00fe
:10bd00000603e900050343004333de000002eb00b5
:10bd1000010037000b0378004822dd00ec457b0072
:10bd20008b85fb00048275008605e9008a0f5300ad
:10bd3000f8ff3e00e08f5400010032000922de00cf
:10bd4000efcf530014003e008784fb000943dd0061
:10bd50000603e9000602620073439000e04f5300bf
:10bd60000d00320016002000e1cf53000200360023
:10bd70000903e9000643dd00860343008703e90069
:10bd80000403630002003a00070262000200370069
:10bd90008783ea000702720004197800534290007a
:10bda0000482fb00848242008100e800634290002c
:10bdb0000482fb00848f5000cdff390014c0b30013
:10bdc000010037000c427800044078004f067800ec
:10bdd0004f05be004f04be0000000600d4c8bf00df
:10bde000000006000200fa00889fbe008a1f78004b
:10bdf000004578008204780024072000848f5000da
:10be00001900320009003e006c025200848f50007d
:10be1000280132006b024200848f5000070032007c
:10be2000e08f500023013200ff003700640720003c
:10be3000848f5000fc003e001e013700e0482a00bd
:10be4000b2040700a99320009944780018c0b300f9
:10be50008acf5400f5003a00f9003700c0492a00a3
:10be6000aa040700f00037003ac9bf008a4f50000b
:10be7000faff3a00fd003700204b2a00a304070018
:10be800099007800814a880079429000e04f520082
:10be90008d003a00f453800094029000858f50008a
:10bea00089003a00144990000281fb008449900007
:10beb000004a800061f8070000047800184a8800f2
:10bec000e00f54000f003200f04c2a008f040700ee
:10bed000104a8000bb040700804e2a008b04070034
:10bee0003ac9bf00d6fc070060c5b30046e9b700f9
:10bef00090c0b30047e9b7006022b8000001eb0032
:10bf000064003700b04e2a00800407006022b800a9
:10bf100008017800912520003ac9bf00940307006a
:10bf2000e04f5000020032004489a8001a00370098
:10bf3000f4538000844a90008582fb009494200092
:10bf4000144278000482fb000402e900848f52004e
:10bf500011003a00244a80004422de00614262005f
:10bf60000d003a00b0512a00680407003ac9bf002a
:10bf7000b3fc070060c5b30046e9b70090c0b3004a
:10bf800047e9b7006022b8000801780011262000b8
:10bf90003ac9bf0076030700004a8000cadb0700e9
:10bfa0004029ef00f453800014047800f85388000f
:10bfb000e00f54002900320098029000e08f5200f8
:10bfc0000d00320005007800c5bf9f0030db070080
:10bfd000004a8800cfba9700e00f500006003a00f0
:10bfe000b0532a004904070050c0b30046e9b70027
:10bff00094c0b30016003700084a9000b6932000a2
:10c0000016437800861f780017c0b300064a8000e8
:10c010000482fb000320220062c0b30011c8b300f9
:10c020003ac9bf00feeb07008f87e90024c0b300c8
:10c03000e04f50000600320000552a00330407008c
:10c04000004a8000a0db07004029ef00990037007c
:10c050000440780047e9b70096003700244a800082
:10c060004422de00614262000c003a0000572a00c0
:10c07000260407003ac9bf0071fc070060c5b30081
:10c0800046e9b70090c0b30047e9b7006022b800a6
:10c0900008017800112620000800370060592a00a6
:10c0a0001a04070040c0b30047e9b700640020004d
:10c0b0000500200062932000f12520003ac9bf004e
:10c0c0002b0307007b0037008040eb003ac9bf001c
:10c0d00024e5070077003700a89420001844780072
:10c0e000e14f54001a003a00e940900024952000e6
:10c0f0001442780084cf500015003a007945900032
:10c10000e04f550008003200f14f55002400320086
:10c110000a40780046e9b70040c0b30047e9b700dd
:10c120004a69ef00410037000ee5070099047800e6
:10c13000894a88000a40780046e9b70040c0b30049
:10c1400047e9b7000a4078004ae9b70037003700ee
:10c1500018c0b3006495200014427800884f520044
:10c1600032003a00e9429000e49520001442780041
:10c1700084cf52002d003a00505b2a00e3030700f1
:10c1800079459000e04f550012003200f14f550004
:10c190000a003a00e1952000914078003ac9bf00ba
:10c1a000f0e4070040c0b30048e9b7004429a80004
:10c1b0000040eb0038fc07001c0037000a40780004
:10c1c00046e9b70040c0b30047e9b7005669ef0041
:10c1d00016003700e1952000914078003ac9bf0071
:10c1e000e0e4070099047800e94a88000a407800f2
:10c1f00046e9b70040c0b30047e9b7000a407800fd
:10c2000056e9b70009003700805c2a00bf03070029
:10c210007940900046e9b7004429a9000040eb00ae
:10c220001dfc0700230037000044eb0008407800a5
:10c230004f0578004f04be000080fa0000000600a1
:10c240001400200005002000a293200001262000f9
:10c2500009407800c602070009407800f8fb070093
:10c260003a69ef004769ef00f0ff3700749420004f
:10c27000144278000482fb00050020006202520094
:10c28000e0825a00e70f5200e08f5a00e6ff3e00be
:10c2900004600100f8fe3700e3ff37008eff37002f
:10c2a000e1ff3700e0ff3700d7ff3700deff370040
:10c2b0000000370018c0b300dcff370010c0b30027
:10c2c00000000600889fbe008a9fbe008c9fbe00b3
:10c2d00000447800a49320001442780010c0b300fa
:10c2e000884f5200970032000040eb00804f520010
:10c2f00094003a00970037000902450094429000ec
:10c30000e4cf520057003a0054429000e34f5200ed
:10c3100002003200e04f520052003a000d40780017
:10c3200045e9b700a000200059da0700e00f5000ef
:10c3300084003200e4538000e00f520004003a0011
:10c34000e0538800f05388000408780004003700a8
:10c35000f4538000000a7800f05388000008eb00d6
:10c36000f453800089024500a5429000054a9800d8
:10c37000eac27c008582fb00858444008902450076
:10c38000154390008c4f530036003a0055439000ff
:10c39000e04f530033003200054b90004833dd007e
:10c3a000f54290008582fb0085027300150298001b
:10c3b000eac27c008582fb00898442008042eb0057
:10c3c000854378000543780010003700b0429000a4
:10c3d000e3cf52000a003a00a0429000e0cf5200a2
:10c3e00004003d00e04f530005003a00054378008b
:10c3f00003003700e0cf530001003a008543780086
:10c40000eac27c000580fb008084440009004500ee
:10c4100090409000e5cf5000ecff32008582fb0099
:10c4200085845400e04f53000e003200084078002d
:10c430003ae9b700664298007742980089024500c1
:10c44000d5439000c83bdd00454390000683fb00c8
:10c450000683730026029800e5429000154a980072
:10c460001bc0b3006ac27c000482fb0084844400c9
:10c47000aa4290008582fb003a4290004822dd00eb
:10c4800005027200848f54009bff3900e0cf5500f5
:10c490002b003200e8538000f85388001802900007
:10c4a000e00f520009003200004a8000e00f500007
:10c4b0000100320084da070018009000f4d9070068
:10c4c000004a8800e00f50001e003200084a900029
:10c4d000b593200095427800851f780017c0b300ff
:10c4e000064a8000980290000482fb00032022008c
:10c4f00062c0b30011c8b3003ac9bf00c8ea070060
:10c50000804278008f87e900e0cf520005003200ba
:10c51000004a80006cda07004029ef000040eb0081
:10c520000800370020c0b30047e9b7000540780095
:10c530004ae9b70056e9b70010c0b3000100370060
:10c540000b4078004f06be004f05be004f04be00f2
:10c5500000000600d453800044a9a900044b9000b9
:10c560000683fb00944a9000c82add008682720090
:10c57000b5498800a44a90008582fb00344a9000a7
:10c580004822dd0005027200c4498800014078009d
:10c590003be9b700ca5380004a40900049e9b70020
:10c5a0008004eb00894578001dc0b3001cc2b300b5
:10c5b000afff3700c902a800c8e2a800c9c2a8009e
:10c5c000c9e2a800c8a2a800c062a800c082a80052
:10c5d000c882a800c922a8006360a8009660a800cd
:10c5e0008660a90000002700ac20b7009660a80074
:10c5f00000000600c902a800c8e2a800c9c2a8003d
:10c60000c9e2a800c8a2a800c062a800c082a80011
:10c61000c882a800c922a80000000600e14f50000f
:10c6200003003a00c902a900cd02a90000000600db
:10c63000c902a80000000600e14f500007003a00c0
:10c64000c8e2a900cce2a900c9c2a900cdc2a900d4
:10c65000c9e2a900cde2a90000000600c8e2a800d6
:10c66000c9c2a800c9e2a80000000600e14f5000be
:10c6700003003a00c8a2a900cca2a900000006004d
:10c68000c8a2a80000000600c902a90010c0b3009b
:10c69000e2ff0700c8e2a900c9c2a900c9e2a900d7
:10c6a00010c0b300e4ff0700c8a2a90010c0b30087
:10c6b000eeff0700c062a900c462a800c082a90002
:10c6c000c482a800c882a900cc82a800c922a900ff
:10c6d000cd22a80000000600e14f500003003a0000
:10c6e000c922a900cd22a90000000600c922a80085
:10c6f00000000600e14f500003003a00c082a9008c
:10c70000c482a90000000600c082a8000000060044
:10c71000e14f500003003a00c882a900cc82a90072
:10c7200000000600c882a80000000600e14f50008b
:10c7300003003a00c062a900c462a900000006001c
:10c74000c062a8000000060064a720001442780020
:10c750000482fb00e5a6200065407a00f3ff070095
:10c7600064a72000144278000482fb0025a7200063
:10c7700065407a00dfff370074a72000144278007c
:10c780000482fb00e5a6200065407a00e0ff070078
:10c7900074a72000144278000482fb0025a7200023
:10c7a00065407a00ccff3700e7ff070065a720004f
:10c7b000954278000042eb00e2cf520001003e00bb
:10c7c0000542e8000440780076eab7000000060061
:10c7d000ddff070065a720009542780034c0b30054
:10c7e000e0cf5200010032000542e9000440780029
:10c7f00076eab70000000600dfff070075a72000fb
:10c800009542780034c0b300e0cf520001003200fe
:10c810000542e9000440780077eab700000006000e
:10c82000d5ff070075a72000954278000042eb0075
:10c83000e2cf520001003e000542e80004407800cb
:10c8400077eab70000000600889fbe0080027800eb
:10c85000020478000502780004f0a7000402ea0050
:10c860000440780006e8b70014c0b300e08f52001f
:10c8700001003c000042eb000440780008e8b700eb
:10c880000102780004f0a7000402ea0004407800e6
:10c8900007e8b70014c0b300e08f500001003c006f
:10c8a0000042eb000440780009e8b700360037008a
:10c8b000e04f5200180032008480200014427800bb
:10c8c000e04f52000a003200c1ff07008004eb0075
:10c8d000040037000014200001002000a503070019
:10c8e0008904e800888f5400faff350009003700fa
:10c8f000adff07008004eb000400370000142000a7
:10c90000010020009b0307008904e800888f540081
:10c91000faff35000668ed007480200014427800ac
:10c92000e04f52001800320094802000144278003a
:10c93000e04f52000a003200afff07008004eb0016
:10c9400004003700001420000100200089030700c4
:10c950008904e800888f5400faff35000900370089
:10c96000afff07008004eb00040037000014200034
:10c97000010020007f0307008904e800888f54002d
:10c98000faff35000768ed0064802000144278004b
:10c990007680200096427200c5ff3a004f04be0028
:10c9a0000000060061006000610260004723dd00b6
:10c9b000f5f72f006716800087826200868272007a
:10c9c000651688004e22dd00f5ff2b0066168000fc
:10c9d0008682620004827200641688004f00dd00c7
:10c9e000f4ff270067168000070262000000720053
:10c9f0006016880000000600caa2ab00feff3a00e5
:10ca000000000600caa2ab00feff320000000600d4
:10ca100002003700caa2ab0002003a00cb02ab0012
:10ca2000fcff3a000000060002003700caa2ab007b
:10ca300002003a00cb02ab00fcff3200000006000f
:08ca4000f3ff0700f8ff3700c7
:020000040000fa
:10ca4800740900006600000000000000da09000018
:10ca58001a000000020000006261f2005e0000009f
:10ca680000000000000301000200000000020000b6
:10ca7800030000000000000002000000780a000027
:10ca88000400000002000000000000000000000098
:10ca9800100a00005e00000000000000000a00000c
:10caa8001000000000000000360900002c00000003
:10cab800000000007c0a00000400000000000000e4
:10cac800d20800006400000002000000000000001e
:10cad800000000000000000000000000000000004e
:10cae800000000000000000000000000000000003e
:10caf800000000000000000000000000000000002e
:10cb0800000000000000000000000000000000001d
:10cb1800000000000000000000000000000000000d
:10cb280000000000000000000000000000000000fd
:10cb380000000000000000000000000000000000ed
:10cb480000000000000000000000000000000000dd
:10cb580000000000f40900000c00000002000000c2
:10cb680000000000000000000000000000000000bd
:10cb780000080000d2000000000000006209000068
:10cb88001200000002000000f3a6010000000000ef
:10cb9800010000000000000000000a000000000082
:10cba800800a000002000000000000006e0a000079
:10cbb8000a0000000200000000000100010001005e
:10cbc8000100030003000000720b000010000000c9
:10cbd80000000000220b00002a00000002000000f4
:10cbe80030313200333435003637380039414200ad
:10cbf80043444500460030003132330034353600b6
:10cc080037383900616263006465660000286e0089
:10cc1800756c6c0029000000820a0000a00000006a
:10cc280002000000010000000000000000000a00ef
:10cc38000000000000000000006400000000000088
:10cc480000000000e80300000000000000001000e1
:10cc5800270000000000000000a08600010000007e
:10cc68000000000040420f000000000000008000ab
:10cc780096980000000000000000e100f5050000a3
:10cc88000000000000ca9a003b00000000000000fd
:10cc9800e40b5400020000000000e800764817008a
:10cca800000000000010a500d4e80000000000000b
:10ccb800a0724e0018090000000040007a10f3002e
:10ccc8005a0000000080c600a47e8d00030000000a
:10ccd80000c16f00f2862300000000008a5d780022
:10cce8004563010000006400a7b3b600e00d000032
:10ccf80000e889000423c7008a000000820b0000b6
:10cd080006000000000000004c0b00002600000098
:10cd180002000000830b000000830b0009000000e4
:10cd280000020000850b000000850b000e020100c8
:10cd380000000000000000000000000006020200e1
:10cd4800000000004c0b0000880b000002000000ef
:10cd580002000000010000008a0b00000200000031
:08cd68000000000000000000c3
:020000040000fa
:10cd7000a4062000848f500007003c000402e90054
:10cd8000848f50000e003d0064025200848f5000da
:10cd90000e003a000a003700c4062000848f5000bd
:10cda0000a00350064024200848f50000400340001
:10cdb00094252000848f500004003a0002003700c0
:10cdc00010c0b30000000600f5ef37000040eb0094
:10cdd000000006000400fa00e0bf9f00f1bf9f00c2
:10cde000950180007fba9700940188006fba970080
:10cdf0001483ba00860078001400ba0095018800f8
:10ce00000080fa0000000600404e200001002000d3
:10ce1000f0ff070074c3b300804f52001a003a00bd
:10ce2000604e200001002000eaff0700d4c2b300da
:10ce3000804f520014003a00804e20000100200074
:10ce4000e4ff070024c6b300804f52000e003a00f2
:10ce5000a04e200001002000deff070094c6b300b2
:10ce6000804f520008003a00c04e20000100200010
:10ce7000d8ff070044c7b300804f520002003a00b9
:10ce8000406e2a00a100070000000600881f7800fd
:10ce900020002000e6010700b8cab300804f54000c
:10cea0001c003200b10a200020002000f801070019
:10ceb00020002000de010700804f54000a003a00e5
:10cec000110020000000eb00f1010700110020001c
:10ced00040002000ee010700a100200060002000bb
:10cee000eb0107000b0037002000200016020700ae
:10cef00000602a00e10020001e0207002000200040
:10cf00000d02070000602a00e1002000190207005e
:10cf1000f5ff37004f047800000006000000eb002a
:10cf2000c3010700cf80de00204b8800314b880012
:10cf3000e20f5000e08f5800040036006429ef0033
:10cf40006629ef006000b800d1010700240020002e
:10cf5000444b88006a29ef0060002000b4010700fc
:10cf6000cf80de00804b8800914b8800800020003d
:10cf7000af010700cf80de00604b8800714b880056
:10cf8000e10f5000e08f5800030036008000eb00f6
:10cf900080002000be01070080002000a4010700df
:10cfa000cf80de00604b8800714b880000000600d7
:10cfb0002ca3ef0020002000ea0107002000200041
:10cfc000dd01070000402c0091002000e90107006e
:10cfd00020002000dc01070000402c009100200010
:10cfe000e401070020002000d301070000402c00ce
:10cff00091002000df01070020002000d20107007f
:10d00000c022a800c9a2a900cda2a90004fe2f0039
:10d0100035358000050262009400b3003435880085
:10d02000f40f2e00653680000502620005502000d6
:10d0300005027200643688001e00070068c0a80060
:10d0400068e0a80000802400811e20004c01070039
:10d050006dff07008dff0700b0ff070010002000e4
:10d06000980107006000b800cae10700bfee0700a2
:10d0700050fd0700104b80002400070080e40700eb
:10d0800093f90700c0ee0700fcff370010c0b300a3
:10d0900000000600040024003604800086026200be
:10d0a000e08f5200fcff3200b011800087c0a90061
:10d0b0000000060024022000c41188000002eb00da
:10d0c000841188003062a8009411880031e2a80021
:10d0d0003342a80087c0a900000006000000240019
:10d0e0008600b6000000ea004f00de0000000600e7
:10d0f0000000fb00a01188000000000000000000fc
:10d100003302ab00feff320000000600881f7800eb
:10d110000004780001003700f5ff07003840780070
:10d12000e04f5000fcff3a004f047800000006007a
:10d13000881f7800004478000042eb0035c6b30039
:10d14000854f5400070036000880fb00440620008d
:10d15000110009000480d8000043b000e4ff07007c
:10d1600014c0b3000884fb0045062000110009002c
:10d170000584d80001447800e94f540002003e00c5
:10d18000e14f520006003a000880fb00a400200096
:10d19000110009000480d8000043b000d4ff07004c
:10d1a0000884fb00a4002000110009000484d800ba
:10d1b00004c3b30004c04000cdff07004f04780053
:10d1c00000000600889fbe008004780044cade008c
:10d1d0006f02620008742a0068407a00c4ff0700ea
:10d1e000ef84640068c07c00c1ff07004f04be00ec
:10d1f00000000600889fbe00800478004c4ade00d4
:10d2000008742a0068407a00b9ff0700484ade0027
:10d210006f02620068407a00b5ff0700444ade00f2
:10d220006f02620068407a00b1ff0700ef8464007b
:10d2300068c07c00aeff07004f04be00000006007f
:10d24000889fbe008a9fbe000005be004c0ade001b
:10d250000500200008742a0068407a00a4ff070037
:10d26000485ade0005002000f90020000482640016
:10d2700068407a009eff0700445ade000500200047
:10d280000482640068407a0099ff07000b82640002
:10d2900068407a0096ff0700445bdd004c52de00d8
:10d2a00004027300cc5ade000482640068407a00f5
:10d2b0008fff0700485bdd004852de000402730068
:10d2c000c85ade000482640068407a0088ff0700c4
:10d2d0004c5bdd004452de0004027300c45ade00e1
:10d2e0000482640068407a0081ff07000a856400b8
:10d2f00068407d007eff07004f05be004f04be0062
:10d30000000006000042eb0065c6b300854f5000e8
:10d3100015003c00e6c25200854f50000200340068
:10d3200094cab3000f00370065c4b300854f5000a6
:10d330000d003c00e6c25200854f50000200340050
:10d3400094ccb3000700370095c3b300854f50005d
:10d3500005003c00eac25200854f50000200340034
:10d3600004cdb300044240000440780000000600f1
:10d370006f406000e94f5000020034007043b0007d
:10d38000000006000043b000000006003222ab009f
:10d39000010032003222a9000000060000037800dc
:10d3a000a4c0b3000040eb0045972000a2c0b3002a
:10d3b0000440bc00e5037900868f530002003a0068
:10d3c000028142000009eb000040e8000442e9004d
:10d3d000f6ff3a0000000600000278000203be00db
:10d3e000d8c9bf0016003200a5c0b3000040eb0052
:10d3f000a2c0b3000440bc0041972000e1017900c5
:10d40000e08f51000a003a00843079000182e80080
:10d4100002024200068abe0066824000020142000b
:10d420000009eb003211780010c0b30000000600c4
:10d430000040e8008542e900edff3a000540780031
:10d4400000000600e00f500003003200e10f500022
:10d4500016003a00120037004497200031000900fe
:10d46000001aeb00440580000400a0000410a10095
:10d470000420a100440588008500a9005008880008
:10d4800004d027007408880004002a00940888004b
:10d490009500a80010c0b300d8e9b700000006004e
:10d4a0009500a900d869ef00000006000040eb00dd
:10d4b000000006003600f800809fbe00829fbe007c
:10d4c000849fbe00869fbe00889fbe008a9fbe00cc
:10d4d0008c1f78003400f80000002000a0018800b4
:10d4e000a9c0b3008045eb004897200066054400c2
:10d4f0000b407800a2c0b3000440bc006802790071
:10d50000e00f520010003200e602410085024400a4
:10d51000100020000100200035034000a5834800d2
:10d5200002064500068ebe000281e80002014400aa
:10d53000b20f5300a28f5b0003003a000400010009
:10d54000000eeb003c1678008b45e8008944e900aa
:10d55000e7ff3a008500a9003400f9004f06780083
:10d560004f05be004f04be004f03be004f02be0079
:10d570004f01be004f00be003600f900004006001b
:10d5800002502300c3002000a2d507008000e9005c
:10d59000f0272d008ed507004ed507000403280084
:10d5a000240888000021ef003406200005088000d0
:10d5b000848f5200fdff360000000600889fbe00e9
:10d5c0008a9fbe000005780047d4de006e04640028
:10d5d000080ab300890c20000b00280085d507003d
:10d5e0003cd507000840780064d5070039d507000e
:10d5f000c510800005826500e00f52000500320072
:10d6000080d5070033d507008904e900f3ff3a000d
:10d610000084eb000a40780058d507002dd507009c
:10d62000080078004f05be004f04be000000060051
:10d63000889fbe00e1ff07000004780071d5070055
:10d6400024d507006bd5070022d507000840e80065
:10d650004ad507001fd507003bd507000084fb0013
:10d6600017d507001bd5070037d507008044780081
:10d6700052d5070017d5070062d5070015d507005a
:10d680004848dd00080070004f04be00000006009e
:10d69000881f780001047800c8ff07000840780060
:10d6a00036d507000bd5070048c0de0033d507008c
:10d6b00008d5070053d5070006d507004f047800aa
:10d6c00000000600881f78000004780044a7a80026
:10d6d000e00f540006003a0020002000210007005f
:10d6e00020002000140007000800780055ff070004
:10d6f0004f047800000006003600f800809fbe004e
:10d70000829fbe00849fbe00869fbe003400f8004a
:10d7100000002000a0018800fae807003400f900aa
:10d720004f03be004f02be004f01be004f00be00bf
:10d730003600f90000400600e20f500001003a00f8
:10d74000c202a80000000600e20f500001003a00eb
:10d75000c202a90000000600000006000040eb0025
:10d7600000000600e20f500001003a00c002a900cc
:04d7700000000600af
:020000040000fa
:10d77400f03fb1000180b10006003500ee0309005e
:10d7840000000000403fb1000180b100fbff3d00fc
:10d794001000b000203fb0000200350000800900f6
:08d7a400000000000000060077
:020000040000fa
:08d7ac000040da000000fe005d
:020000040000fa
:020000040001f9
:0457f00033ff000083
:020000040000fa
:020000040001f9
:0457f400c0f40000fd
:020000040000fa
:020000040001f9
:0457f8008f09000015
:020000040000fa
:020000040001f9
:0457fc00601f00002a
:00000001FF
